:100000000C941F080C9449080C9449080C94490856
:100010000C9449080C9449080C9449080C9449081C
:100020000C9449080C9449080C9449080C9449080C
:100030000C9449080C9449080C9420100C9449081D
:100040000C944B470C9449080C94A94A0C94DF4A31
:100050000C9449080C9449080C9449080C944908DC
:100060000C9449080C9449080C9449080C944908CC
:100070000C9449080C9449080C9449080C944908BC
:100080000C9449080C9461350C9449082A2A2A2AB0
:100090002A2A2A2A2A2A2A2A2A2A2A2A2A2A2A2AC0
:1000A0002A2A2A2A2A2A2A00696E697469616C69D7
:1000B0007A6174696F6E204F4B2E00696E697469A6
:1000C000616C697A6174696F6E206661696C6564E0
:1000D000212048414C5400496E697469616C697A09
:1000E000696E6720534420636172642E2E2E002AAD
:1000F0002A2A2A2A2A2A2A2A207374617274202A18
:100100002A2A2A2A2A2A2A2A2A2A004E6F205344D7
:1001100020636172640054524B20504C4159455247
:10012000005353443133303620616C6C6F6361741B
:10013000696F6E206661696C6564002D2D2D2D2D13
:100140002D2D20656E6420616C6C202D2D2D2D2DA4
:100150002D2D2D2D2D002D2D2D2D2D2D2D20616C96
:100160006C202D2D2D2D2D2D2D2D2D2D2D2D0020C7
:100170002D20656E642020626C6F636B2073656E4A
:100180006400202D206C656E2020626C6F636B0014
:10019000202D20737461727420626C6F636B207306
:1001A000656E64002D2D2D2D2D2D20626C6F636BDF
:1001B0002073656E64202D2D2D2D2D2D2D2D2D2D93
:1001C0002D2D2D00202D20656E6420686561642032
:1001D00073656E6400202D206C656E206865616417
:1001E0002073656E6400202D207374617274206822
:1001F0006561642073656E64002D2D2D2D2D2D2DD0
:100200002D20686561642073656E64202D2D2D2D71
:100210002D2D2D2D2D2D2D00D0B1D183D184D0B5F4
:10022000D18020D0BED0BFD183D181D182D0BED1E8
:1002300088D0B5D0BD002A2A2A2A2A204D454D2033
:100240004C4F4144204252552A2A2A2A2A002A2A5F
:100250002A2A2A2073694D454D204C4F4144202ABB
:100260002A2A2A2A00200020002000000000000086
:1002700000000000000000640064006400DB000077
:10028000000000000000000000190000009B009B1F
:10029000009B009B009B009B009B009B009B009B86
:1002A00000000002000100FF00FF000000282328DA
:1002B000231C25530684038403F02300000F27E743
:1002C000030100E703E703E703E703E703E703E7C7
:1002D00003E703E703E70300000000010096008046
:1002E000000000E803E803AC0D6B02BE00C900F497
:1002F000000000AC0DC7010100C701C701BC02C767
:1003000001C701C701C701C701C701C70197048A17
:10031000047D04700463045204450438042B041E55
:100320000411040404F703EA03DD03D003C303B696
:1003300003A9039C038F038203750368035B034EC9
:100340000343034E6F2053442063617264004544AD
:100350004D20646174612075733E005253532064D4
:100360006174612075733E0042534D206461746175
:100370002075733E00524B4920646174612075738F
:100380003E00524B5320646174612075733E0052ED
:100390004B4120646174612075733E00524B4D20C7
:1003A000646174612075733E00524B502064617427
:1003B000612075733E00524B4F206461746120755B
:1003C000733E00524B2073796E63206164643E007B
:1003D000524B2020646174612075733E00524B20A3
:1003E00070696C6F742075733E005A582073706585
:1003F0006564202D2D3E005A5820646174612020D0
:1004000075733E005A582073796E63322075733EBF
:10041000005A582073796E63312075733E005A5824
:100420002070696C6F742075733E005A5820706993
:100430006C6F74206C656E005A58207061757A324A
:100440002075733E005A58207061757A612075736B
:100450003E0053455420414C4C2044454641554CA8
:10046000543F004C4544204C4344206F6E203E00D6
:100470004265657020766F6C756D653E00426565FE
:1004800070206F6E5F6F66663E004D4F4445205092
:100490004C41592D2D3E0045584954206D656E75CF
:1004A0002D3E3E3E2F2E2E007D0570056305560520
:1004B0004705380528051A0510050505F704EA045F
:1004C000DE04D104C6044E4F20534420434152441D
:1004D00000494E495420534420434152440044456E
:1004E0004641554C54205345540044454641554CD3
:1004F0005420414C4C3F0044454641554C542054F7
:100500004849533F0054524B3A20504155534500FF
:1005100054524B3A2053544F5000534156454420B7
:100520004550524F4D202A0054524B3A20534554C7
:100530005550204D454E550054524B3A205A5820A4
:10054000424C4F434B3A0054524B3A204D6F646536
:100550002D4D4943520054524B3A204D6F64652D46
:100560004F520054524B3A204D6F64652D524B0050
:1005700054524B3A204D6F64652D5A580054524BDB
:100580003A204D6F64652D4155544F007C3C3E5ED2
:100590002B3D3F2F5B5D3B2C2A225C0000000000BE
:1005A000003E5B4F5B3E3E6B4F6B3E1C3E7C3E1CF9
:1005B000183C7E3C181C577D571C1C5E7F5E1C003F
:1005C000183C1800FFE7C3E7FF0018241800FFE7F6
:1005D000DBE7FF30483A060E2629792926407F05B9
:1005E0000507407F05253F5A3CE73C5A7F3E1C1CCF
:1005F00008081C1C3E7F14227F22145F5F005F5F8F
:1006000006097F017F006689956A6060606060947A
:10061000A2FFA29408047E040810207E201008087F
:100620002A1C08081C2A08081E101010100C1E0C8A
:100630001E0C30383E3830060E3E0E06000000001C
:100640000000005F00000007000700147F147F1403
:10065000242A7F2A12231308646236495620500048
:1006600008070300001C2241000041221C002A1C34
:100670007F1C2A08083E080800807030000808081F
:100680000808000060600020100804023E5149453F
:100690003E00427F400072494949462141494D335D
:1006A0001814127F1027454545393C4A49493141C4
:1006B000211109073649494936464949291E000092
:1006C00014000000403400000008142241141414E7
:1006D0001414004122140802015909063E415D59D3
:1006E0004E7C1211127C7F494949363E41414122DC
:1006F0007F4141413E7F494949417F090909013E06
:10070000414151737F0808087F00417F410020402C
:10071000413F017F081422417F404040407F021C3E
:10072000027F7F0408107F3E4141413E7F09090955
:10073000063E4151215E7F09192946264949493221
:1007400003017F01033F4040403F1F2040201F3FE7
:100750004038403F6314081463030478040361596C
:10076000494D43007F4141410204081020004141AE
:10077000417F04020102044040404040000307085A
:100780000020545478407F28444438384444442856
:10079000384444287F385454541800087E090218FD
:1007A000A4A49C787F0804047800447D4000204085
:1007B000403D007F1028440000417F40007C0478C9
:1007C00004787C080404783844444438FC18242411
:1007D0001818242418FC7C08040408485454542491
:1007E00004043F44243C4040207C1C2040201C3C0E
:1007F0004030403C44281028444C9090907C446405
:10080000544C440008364100000077000000413697
:10081000080002010204023C2623263C1EA1A1611D
:10082000123A4040207A385454555921555579414F
:100830002254547842215554784020545579400C24
:100840001E52721239555555593954545459395507
:100850005454580000457C410002457D420001454A
:100860007C407D1211127DF0282528F07C545545DE
:10087000002054547C547C0A097F4932494949324A
:100880003A4444443A324A4848303A4141217A3A5B
:1008900042402078009DA0A07D3D4242423D3D4027
:1008A00040403D3C24FF2424487E4943662B2FFCD6
:1008B0002F2BFF0929F620C0887E09032054547984
:1008C000410000447D413048484A32384040227A55
:1008D000007A0A0A727D0D19317D2629292F2826D2
:1008E0002929292630484D402038080808080808DA
:1008F0000808382F10C8ACBA2F102834FA00007B33
:10090000000008142A142222142A14085500550045
:1009100055AA55AA55AAFF55FF55FF000000FF0034
:10092000101010FF00141414FF001010FF00FF102F
:1009300010F010F0141414FC001414F700FF000061
:10094000FF00FF1414F404FC141417101F10101FE0
:10095000101F1414141F00101010F0000000001FCE
:10096000101010101F10101010F010000000FF10D9
:100970001010101010101010FF10000000FF1400D5
:1009800000FF00FF00001F10170000FC04F4141407
:100990001710171414F404F40000FF00F7141414D3
:1009A00014141414F700F7141414171410101F1053
:1009B0001F141414F4141010F010F000001F101F76
:1009C0000000001F14000000FC140000F010F010E4
:1009D00010FF10FF141414FF141010101F0000005B
:1009E00000F010FFFFFFFFFFF0F0F0F0F0FFFFFF5F
:1009F0000000000000FFFF0F0F0F0F0F38444438B6
:100A000044FC4A4A4A347E02020606027E027E0204
:100A100063554941633844443C04407E201E20060F
:100A2000027E020299A5E7A5991C2A492A1C4C724C
:100A300001724C304A4D4D303048784830BC625AD3
:100A4000463D3E494949007E0101017E2A2A2A2A63
:100A50002A44445F444440514A444040444A51403F
:100A60000000FF0103E080FF000008086B6B083600
:100A700012362436060F090F060000181800000071
:100A80001010003040FF0101001F01011E00191D60
:100A90001712003C3C3C3C00000000002200FF21FB
:100AA00000000103070F1F3F7F0080C0E0F0F8FC4B
:100AB000FEDB40A4A62EAF2000A1C8D300408DAE1F
:100AC000D580A800006000000000000000000000C9
:100AD00000000000E0000000000000000000000036
:100AE000000001E000000000000000000000000025
:100AF0000001F00000000000000000000000000005
:100B000003F00000000000000000000000000007EB
:100B1000F00000000000000000000000000007F8E6
:100B2000000000000000000000000000000FF800BE
:100B3000000003C0007E000001E0007F0FF800000D
:100B40000003C000FE000001E000FFEFF80000001D
:100B500003C000FE000001E000FFFFF800000003FA
:100B6000C000F00000000F007FFE7FC0000003C047
:100B700000F00000000F003FFE7FF83FF1FBCFFCCC
:100B8000FEF3BC3DEFE01FFE7FFF7FFBFFDFFEFEBD
:100B9000FFBC3DEFE01FC6FFFF7FFBFFDFFEFEFF58
:100BA000BC3DEFE00FE3C7FE787BC3DE1EF0FFBC69
:100BB0003DEF0007FF87FC787BC3DE1EF0F83C3D6D
:100BC000EF0001FFFFF0007BC3C01EF0F03C3DEFE3
:100BD0000001F37FE03FFBC3CFFEF0F03C3DEF00B0
:100BE00003E33F807FFBC3DFFEF0F03C3DEF0007F7
:100BF000E73C00787BC3DE1EF0F03C3DEF0007FFD2
:100C0000BE00787BC3DE1EF0F03C3DEF0007FFFE28
:100C100000787BC3DE1EF0F03C3DEF000FFFFE00CE
:100C20007FFBFFDFFEF0F03FFDEFE00FFFFF007FF7
:100C3000FBFFDFFEF0F03FFDEFE00FF9FF003E7934
:100C4000F9CF9EF0F01F3DE7E01FF1FF000000002C
:100C500000000000000000001F80FF007FFFFFFF7A
:100C6000FFFFFFFFFFFFE01C007F007FFFFFFFFE95
:100C7000B46D888D18E000001F007FFFFFFFFE9518
:100C8000AD7DB577E000000F007FFFFFFFFEA5AD53
:100C90009D8D19E0000006007FFFFFFFFEB5ADED62
:100CA000B57EE000000000000180000000000000B0
:100CB000000000038000000000000000000007C0EA
:100CC00000000000000000000007C000000000005D
:100CD000000000000FC00000000000000000001F26
:100CE000E00000000000000000001FE00000000025
:100CF00000000000003FE0000000000000000000D5
:100D00003FF00000000000000000007FF000000045
:100D1000000000001FF87FF0000000000000003F0E
:100D2000FE7FF0000000000000003FFF7FF00000A9
:100D300000000000001FFFFBE000000000000000BA
:100D40000FFFF9FFC00000000000000FFFF9FFF8DF
:100D500000000000000007FFF1FFFF00000000009E
:100D60000003FC73FFFF80000000000001FE3FFF56
:100D7000FF80000000000000FF1E0FFF00000000C9
:100D80000000007FFE1FFC000000000000003FFF8D
:100D9000FFF8000000000000000FDFFFE00000008F
:100DA000000000001F19FFC0000000000000003F0D
:100DB0003CFF00000000000000007E7CF800000006
:100DC00000000000007FFE7C00000000000000002A
:100DD000FFFFFC0000000000000000FFFFFE00001D
:100DE000000000000000FFFFFE0000000000000007
:100DF00001FFEFFE0000000000000001FFCFFE0039
:100E000000000000000003FF07FE000000000000DB
:100E10000003FC07FE0000000000000003F003FEDA
:100E200000000000000000018000FE000000000043
:100E300000000000007E0000000000000000000034
:100E40003E000000000000000000000C0000000058
:100E50000000078000FC000003C0000000078001C4
:100E6000FC000003C0000000078001FC000003C07C
:100E7000000000078001E00000001E000000078065
:100E800001E00000001E007FE3F79FF9FDE7787B9B
:100E9000DFC0FFF7FFBFFDFDFF787BDFC0FFF7FF7F
:100EA000BFFDFDFF787BDFC0F0F787BC3DE1FF7839
:100EB0007BDE00F0F787BC3DE1F0787BDE0000F7D9
:100EC00087803DE1E0787BDE007FF7879FFDE1E0F2
:100ED000787BDE00FFF787BFFDE1E0787BDE00F086
:100EE000F787BC3DE1E0787BDE00F0F787BC3DE1B1
:100EF000E0787BDE00F0F787BC3DE1E0787BDE0048
:100F0000FFF7FFBFFDE1E07FFBDFC0FFF7FFBFFDA5
:100F1000E1E07FFBDFC07CF3F39F3DE1E03E7BCF70
:100F2000C00000000000000000000000FFFFFFFF05
:100F3000FFFFFFFFFFFFC0FFFFFFFFFD68DB111A90
:100F400031C0FFFFFFFFFD2B5AFB6AEFC0FFFFFF21
:100F5000FFFD4B5B3B1A33C0FFFFFFFFFD6B5BDB0D
:100F60006AFDC00000000A0B0C0000000000000138
:100F70000405060000000000000000000000000062
:100F80000000000000000000000000000000000061
:100F90000000000000000000010204081020408052
:100FA00001020408102040800810010204081020EB
:100FB000408001020102040810204080048040208B
:100FC00010080402010102040810204080050505F4
:100FD00005050505050202020202020202070704D6
:100FE00004040404040404070703030303030303C2
:100FF00003070101010101010101060606060606BB
:1010000006060000390036003300300021002000C1
:10101000630000003B00380035003200230062000E
:10102000650000003A003700340031002200610002
:101030006400BE1D9F21D4249134134B261E11241D
:101040001FBECFEFD0E1DEBFCDBF12E0A0E0B1E028
:10105000EAEFFAEA00E00BBF02C007900D92AE3B48
:10106000B107D9F728E0AEEBB2E001C01D92A9317B
:10107000B207E1F718E0CEE1D8E004C02197FE0105
:101080000E94B04FC931D107C9F70E947E4F0C941E
:1010900070550C94000090E080E008950895FF9250
:1010A0000F931F93CF93DF938C01EB01F8800E9485
:1010B0005B55F81621F06F2DC8010E946355CE01D3
:1010C000DF91CF911F910F91FF900895CF93DF9300
:1010D000EB010E945B558883CE01DF91CF9108958B
:1010E0000F931F93CF93DF9300D0CDB7DEB7082FB8
:1010F00010E0000F111FF801E35FFB4F8081918129
:101100009A838983BE016E5F7F4FC8010E944F089A
:10111000BE016F5F7F4FC80101960E944F080F907C
:101120000F90DF91CF911F910F9108950F931F930F
:10113000CF93DF9300D0CDB7DEB7082F10E0000FBC
:10114000111FF801E952FD4F85919491F801E35F79
:10115000FB4F808391839A838983BE016E5F7F4FAB
:10116000C8010E944F08BE016F5F7F4FC801019602
:101170000E944F080F900F90DF91CF911F910F9118
:101180000895EF92FF920F931F93CF93DF9300D0B8
:10119000CDB7DEB7082F000F10E0812F869590E0C5
:1011A000880F991FFC01E952FD4F25913491FC01F4
:1011B000E35FFB4F208331833A832983E12EF12CB7
:1011C000BE016E5F7F4FC7010E944F08BE016F5F77
:1011D0007F4FC70101960E944F081E5F0117E8F676
:1011E0000F900F90DF91CF911F910F91FF90EF9093
:1011F0000895EF92FF920F931F93CF93DF9300D048
:10120000CDB7DEB7082F000F10E0E12EF12CBE01A4
:101210006E5F7F4FC7010E946608BE016F5F7F4F00
:10122000C70101960E94660869818A810E94864CE6
:10123000E12FE695F0E0EE0FFF1FE35FFB4F918398
:1012400080831E5F011708F70F900F90DF91CF91F9
:101250001F910F91FF90EF90089561E08BED93E067
:101260000E94EB3161E084EC93E00E94EB3161E09D
:101270008DEA93E00E94EB3161E086E993E00E9401
:10128000EB316CED75E086E993E00E9489316FE007
:1012900070E084EC93E00E948D316FE070E08DEAA5
:1012A00093E00C948D318FB90000779BFECF8FB106
:1012B0000895CF92DF92EF92FF920F931F93CF93F7
:1012C000DF93CDB7DEB762970FB6F894DEBF0FBEDF
:1012D000CDBFE82EF62E8A018FE00E944149892B6E
:1012E00041F088E19FE00FB6F894A89581BD0FBE4C
:1012F00091BDB801CE010D960E94F24DEE2DF0E0A9
:10130000EE0FFF1FE855FB4F65917491CE010796D4
:101310000E94244E64EC71E0C8010E94AF4E882305
:1013200081F0EF2DF0E0EE0FFF1FE35FFC4F6591C2
:101330007491C8010E940A4EB801CE010D960E9418
:10134000DB4D85E0E81212C04AE060915304CE0103
:1013500001960E941B4DBE016F5F7F4FCE01079625
:101360000E94594ECE0101960E948A4C80916E04D3
:101370008823B1F1F801848195810E9788F5E09179
:101380005604F0E0EE0FFF1FE35FFB4F60817181B9
:101390004AE0CE0101960E94484DBE016F5F7F4F2B
:1013A000C8010E94594ECE0101960E948A4CE091DC
:1013B0005604F0E0EE0FFF1FE35FFB4F6081718189
:1013C0004AE0CE0101960E94484DBE016F5F7F4FFB
:1013D000CE010D960E94594ECE0101960E948A4C74
:1013E00040E060E088E393E00E94614663E371E0DF
:1013F00088E393E00E94AE4B40E060E088E393E036
:101400000E946146BE01695F7F4F88E393E00E94BE
:10141000A04B41E060E088E393E00E94614663E313
:1014200071E088E393E00E94AE4B41E060E088E326
:1014300093E00E946146B80188E393E00E94A04BCC
:1014400088E393E00E94364780916F04882351F02F
:1014500041E06CE088E393E00E94614688E393E01A
:101460000E943D47BE01695F7F4F88E797E00E9479
:10147000D34BB80188E797E00E94D34BBE01635F6E
:101480007F4F88E797E00E94D34B86E593E00E9468
:101490002F4161E086E593E00E94D23E0AE010E031
:1014A000109363030093620386E090E090936503DA
:1014B00080936403BE01695F7F4F86E593E00E94DD
:1014C000A04B109363030093620386E190E0909336
:1014D000650380936403BE01635F7F4F86E593E0FD
:1014E0000E94A04B80916F04882391F0CC24C39478
:1014F000D12C93E0E92EF12C0DE010E02EE130E04C
:1015000043E150E06FE470E086E593E00E944C3ADE
:1015100086E593E00E94C444CE0107960E948A4C5F
:10152000CE010D960E948A4C62960FB6F894DEBFEB
:101530000FBECDBFDF91CF911F910F91FF90EF9024
:10154000DF90CF900895CF93DF9300D000D000D0EC
:10155000CDB7DEB781E080936F0464EC71E0CE011B
:1015600001960E94FC4CAE014F5F5F4F60915604A4
:10157000809157040E945909CE0101960E948A4C1D
:1015800026960FB6F894DEBF0FBECDBFDF91CF9188
:101590000895CF93DF9300D000D000D0CDB7DEB751
:1015A00010926F0464EC71E0CE0101960E94FC4C35
:1015B000AE014F5F5F4F60915604809157040E94C7
:1015C0005909CE0101960E948A4C26960FB6F894CE
:1015D000DEBF0FBECDBFDF91CF910895FF920F9375
:1015E0001F93CF93DF93D62F172FF82EC42F2111DF
:1015F0001AC01F9882E00E945309002319F08F2D12
:101600000E945309812F0E9453098D2F0E94530974
:101610008C2F0E9453091F9A1E9ADF91CF911F9120
:101620000F91FF9008951E98E5CF0F931F93CF93CE
:10163000DF93EB01182F022F411119C01F9883E08F
:101640000E945309002319F0812F0E9453098D2F06
:101650000E9453098C2F0E9453098FEF0E94530957
:101660001F9A1E9ADF91CF911F910F9108951E9896
:10167000E6CF8F929F92AF92BF92CF92DF92EF927E
:10168000FF920F931F93C0900601D0900701E09046
:101690000801F09009018090340390903503A090E8
:1016A0003603B090370397018601080D191D2A1DD6
:1016B0003B1D601771078207930740F56C157D0588
:1016C0008E059F05A8F421E031E0C316D104E3069E
:1016D000F10408F420E040E01F910F91FF90EF909B
:1016E000DF90CF90BF90AF909F908F900C94150B90
:1016F0006C197D098E099F0921E031E08316910460
:10170000A306B10408F420E041E0E6CF8FEF1F917B
:101710000F91FF90EF90DF90CF90BF90AF909F9090
:101720008F900895CF92DF92EF92FF920F93C09027
:101730000601D0900701E0900801F09009016C15B6
:101740007D058E059F0588F401E021E0C216D104D5
:10175000E206F10408F400E020E00E94EE0A0F9196
:10176000FF90EF90DF90CF9008956C197D098E095E
:101770009F0901E0C0903403D0903503E090360318
:10178000F090370321E0C216D104E206F10408F418
:1017900000E021E0E2CF8F929F92AF92BF92CF9272
:1017A000DF92EF92FF920F936B017C0149015A0186
:1017B000C814D904EA04FB0458F4402FC701B60149
:1017C0000E94920B8FEFC81AD80AE80AF80AF0CFE5
:1017D0000F91FF90EF90DF90CF90BF90AF909F90D0
:1017E0008F900895EF92FF920F931F93CF93DF9303
:1017F00000D01F92CDB7DEB78C011F926F9384E4A7
:1018000091E09F938F93CE0101967C019F938F93DC
:101810000E947452B701C8010E94FC4C0F900F90B7
:101820000F900F900F900F90C8010F900F900F9096
:10183000DF91CF911F910F91FF90EF900895CF927C
:10184000DF92EF92FF920F931F93CF93DF9300D01D
:1018500000D01F92CDB7DEB78C016A017B01A701D2
:101860006627772720E130E088E797E00E94484C20
:10187000FF92EF92DF92CF9289E491E09F938F9352
:10188000CE0101967C019F938F930E947452B70101
:10189000C8010E94FC4C0FB6F894DEBF0FBECDBF4E
:1018A000C8010F900F900F900F900F90DF91CF9184
:1018B0001F910F91FF90EF90DF90CF9008954F927E
:1018C0005F926F927F928F929F92AF92BF92CF92D0
:1018D000DF92EF92FF921F93CF93DF9300D000D05F
:1018E00000D0CDB7DEB76B017C0129013A01BC0104
:1018F000A601CE0101960E941F0CBE016F5F7F4FB3
:1019000088E797E00E94A04BCE0101960E948A4C86
:1019100069E672E088E797E00E947C4B1FE04C1478
:101920005D046E047F0408F448C0C701B6010E943C
:10193000390B682FCE0101960E94F20BBE016F5F3A
:101940007F4F88E797E00E94A04BCE0101960E944E
:101950008A4C67E672E088E797E00E947C4B46017C
:1019600057018FEF881A980AA80AB80A111121C0E6
:10197000C414D504E604F704E1F088E797E00E9478
:10198000BD4BB501A401CE0101960E941F0CBE0102
:101990006F5F7F4F88E797E00E94A04BCE010196D2
:1019A0000E948A4C65E672E088E797E00E947C4BD3
:1019B00010E1115075016401B2CF88E797E00E94F1
:1019C000BD4B26960FB6F894DEBF0FBECDBFDF919C
:1019D000CF911F91FF90EF90DF90CF90BF90AF908D
:1019E0009F908F907F906F905F904F9008950F938E
:1019F000CF93DF93C1E0811101C0C0E000E02C2F44
:101A000043E360E070E0CB010E94EE0A2C2F47E731
:101A100061E070E080E090E00E94EE0A20E04C2F50
:101A200060E070E0CB010E94150B833339F56EE462
:101A300071E088E797E00E94E54B20E04C2F60E0E2
:101A400070E081E090E00E94150B833309F450C0F0
:101A5000D0E020E04C2F60E070E880E090E00E9451
:101A6000150B833359F420E04C2F61E070E880E0DF
:101A700090E00E94150B873709F4D1E001E02C2F8C
:101A80004AEA60E070E0CB010E94EE0A2C2F45E5A7
:101A900061E070E080E090E00E94EE0A21E04C2FCF
:101AA00060E070E0CB010E94150B8A3AE1F461E539
:101AB00071E088E797E00E94E54B21E04C2F60E061
:101AC00070E082E090E00E94150B8A3A59F421E020
:101AD0004C2F61E070E082E090E00E94150BD3E0B3
:101AE000853509F0D0E08D2FDF91CF910F910895CA
:101AF00020E04C2F61E070E0CB010E94150B87378E
:101B000009F0A6CFD2E0A5CF61E087E00E94D748D8
:101B100061E086E00E94D74861E087E00E941349B7
:101B200061E086E00E94134980E00E94F70C811179
:101B300016C010920601109207011092080110922F
:101B4000090181E00E94F70C811126C01092340334
:101B500010923503109236031092370308958130A6
:101B600069F480E090E8A0E0B0E0809306019093F3
:101B70000701A0930801B0930901E3CF823029F453
:101B800080E090E0A1E0B0E0F0CF8330D1F680E0DB
:101B900090E0A2E0B0E0E9CF813069F480E090E825
:101BA000A0E0B0E08093340390933503A093360314
:101BB000B09337030895823029F480E090E0A1E0EB
:101BC000B0E0F0CF8330B1F780E090E0A2E0B0E089
:101BD000E9CFEF92FF921F93CF93DF93EC017B014C
:101BE00010E0BE0190E080E00E94390B612F680F89
:101BF000CE15DF0519F02196162FF3CF812FDF9137
:101C0000CF911F91FF90EF900C94864CCF93DF9370
:101C1000FB0122813381DC0113963C932E931297B2
:101C2000448155816681778114964D935D936D93C0
:101C30007C931797408551856285738518964D93DF
:101C40005D936D937C931B971C96EF012C969C01E2
:101C5000275E3F4F49914D93A217B307D9F7218DC6
:101C6000328DFC01328F218FDF91CF910895CF9279
:101C7000DF92EF92FF920F931F93CF93DF93CDB735
:101C8000DEB7E6970FB6F894DEBF0FBECDBF7C017E
:101C9000162F6EE472E088E797E00E94C14BB7010F
:101CA00088E797E00E94D34BCE014C960E94FC1E21
:101CB000F7014081518121E060E774E0CE01019697
:101CC0000E94BE20BE016F5F7F4FCE014C960E94E6
:101CD000060ECE014C960E942C1F6F5F7F4F7093B3
:101CE000500460934F044AE050E088E797E00E9478
:101CF000744CC12CD12C760180914F0490915004EA
:101D0000B0E0A0E0C816D906EA06FB0660F5CE01F1
:101D10004C960E94991E082F1123D1F0C114D104B2
:101D2000E104F104A9F4863E99F046EE60E070E02B
:101D3000CB010E94920B80914F0490915004019628
:101D40009093500480934F04C12CD12C7601C394FE
:101D5000402FC701B6010E94920BFFEFCF1ADF0A96
:101D6000EF0AFF0AC9CFE6960FB6F894DEBF0FBEA2
:101D7000CDBFDF91CF911F910F91FF90EF90DF903A
:101D8000CF9008958F929F92AF92BF92CF92DF92A1
:101D9000EF92FF920F931F93CF93DF93CDB7DEB7F0
:101DA000E6970FB6F894DEBF0FBECDBF8C0166E399
:101DB00072E088E797E00E94C14BB80188E797E09E
:101DC0000E94D34BCE014C960E94FC1EF80140812C
:101DD000518121E060E774E0CE0101960E94BE20AF
:101DE000BE016F5F7F4FCE014C960E94060ECE0162
:101DF0004C960E942C1F6F5F7F4F7093500460932E
:101E00004F044AE050E088E797E00E94744C46EEA9
:101E100060E070E0CB010E94920B09E010E00150FD
:101E2000110999F0CE014C960E94991E682F88E7FF
:101E300097E00E94B64B80914F0490915004019717
:101E40009093500480934F04EACF64EC71E088E7EC
:101E500097E00E94E54BCE014C960E94991E182FE8
:101E6000CE014C960E94991E082F612F0E94864C2D
:101E70006C01402F61E070E080E090E00E94920BE6
:101E8000412F62E070E080E090E00E94920BCE0172
:101E90004C960E94991E182FCE014C960E94991EB6
:101EA000612F0E94864C8C017601E80EF91E64E5D4
:101EB00071E088E797E00E94AE4B40E150E0B60148
:101EC00088E797E00E94744C6FE571E088E797E03F
:101ED0000E94AE4B40E150E0B80188E797E00E94D5
:101EE000744C68E671E088E797E00E94AE4B40E1F1
:101EF00050E0B70188E797E00E94744C4F2D63E0F3
:101F000070E080E090E00E94920B4E2D64E070E063
:101F100080E090E00E94920BCE014C960E94991EA8
:101F2000CE014C960E94991ECE014C960E94991E9D
:101F3000CE014C960E94991E80914F0490915004BE
:101F400009979093500480934F047801F7E0EF0EC7
:101F5000F11C85E0C82ED12C4601B12CA12C8FEFAD
:101F6000C81AD80AEC14FD0451F0CE014C960E9418
:101F7000991E482FC501B4010E94920BEDCF40E09D
:101F8000C501B4010E94920BB70190E080E040E0EF
:101F90000E94920BB801685F7F4F90E080E046EEB0
:101FA0000E94920BB8016B5F7F4F85E090E00E942A
:101FB000E90DF82E492FB801675F7F4F90E080E070
:101FC0000E94920BB801665F7F4F90E080E04F2D3A
:101FD0000E94920B055F1F4F1093500400934F0413
:101FE000E6960FB6F894DEBF0FBECDBFDF91CF915E
:101FF0001F910F91FF90EF90DF90CF90BF90AF9027
:102000009F908F9008951FBC1EBC8EB581608EBDC1
:10201000089587B78B7F87BF0895789487B78460CA
:1020200087BF08958350904F24E0880F991F2A9509
:10203000E1F7809590959093520480935104089510
:102040001F920F920FB60F9211240BB60F922F937F
:102050003F934F935F936F937F938F939F93AF9330
:10206000BF93EF93FF9380915104909152049DBDD3
:102070008CBD80916A0491E0892780936A048091E5
:102080006C04882351F083E00E94414961E0892B70
:1020900009F060E083E00E94134981E080936904C5
:1020A000FF91EF91BF91AF919F918F917F916F9130
:1020B0005F914F913F912F910F900BBE0F900FBEEC
:1020C0000F901F9018950E94091064EF71E080E056
:1020D00090E00E94C74780E30E944149892BD9F7CD
:1020E00064EF71E080E090E00E94C7470C940D100F
:1020F0001092500410924F04809155048093530421
:102100000895CF93C0914304C730D8F4609141043F
:102110007091420490E080E00E94390BEC2FF0E0D7
:10212000EC5BFB4F808380914104909142040196C7
:102130009093420480934104809143048F5F809385
:10214000430480E30E944149892B11F40E946310EB
:102150008DE20E944149892B19F4CF910C9478109B
:10216000CF9108950F931F93CF93DF9300D000D0AA
:1021700000D0CDB7DEB70EE511E08BED93E00E9405
:10218000D232882369F00E94C90A26960FB6F894C5
:10219000DEBF0FBECDBFDF91CF911F910F9108958C
:1021A00086E993E00E94E532882389F110926F045A
:1021B00064EC71E0CE0101960E94FC4CAE014F5FD1
:1021C0005F4F6091560487E00E945909CE01019645
:1021D0000E948A4C809156040E94700860ED77E05E
:1021E00080E090E00E94C74764EC71E0CE01019668
:1021F0000E94FC4CAE014F5F5F4F6091560486E039
:102200000E945909CE0101960E948A4CBECF86E9F0
:1022100093E00E941333882309F447C064EC71E013
:10222000CE0101960E94FC4CAE014F5F5F4F609162
:1022300056048AE00E945909CE0101960E948A4CF8
:1022400086E993E00E94E532882309F451C064ECEA
:1022500071E0CE0101960E94FC4CAE014F5F5F4FD2
:10226000609156048CE00E945909CE0101960E94AB
:102270008A4C809156040E94960860ED77E080E0D9
:1022800090E00E94C74764EC71E0CE0101960E9485
:10229000FC4CAE014F5F5F4F6091560486E00E9498
:1022A0005909CE0101960E948A4C8DEA93E00E9462
:1022B000D232882329F120915604822F90E0880F92
:1022C000991FFC01EF55FD4F45915491FC01E559D3
:1022D000FD4F45915491FC01E35FFB4F808191815B
:1022E0004817590708F037C001979183808335C09C
:1022F0008BED93E00E94D232882309F4A1CFC3CFA3
:1023000060E08DEA93E00E942D338111D4CF84ECFC
:1023100093E00E94D232882309F44FC020915604E2
:10232000822F90E0880F991FFC01EF55FD4F4591DA
:102330005491FC01E559FD4F65917491FC01E35FF7
:10234000FB4F808191818417950708F03EC001966C
:10235000918380833CC051834083243039F4609161
:102360001504709116048CE00E942E4864EC71E014
:10237000CE0101960E94FC4CAE014F5F5F4F609111
:102380005604809157040E945909CE0101960E947B
:102390008A4C0431110514F00A501109B8018DEA74
:1023A00093E00E948D318DEA93E00E94BE32882333
:1023B00009F4ADCF0EE511E0AACF60E084EC93E024
:1023C0000E942D338111AACFD8CE5183408324306F
:1023D00039F460911504709116048CE00E942E4827
:1023E00064EC71E0CE0101960E94FC4CAE014F5F9F
:1023F0005F4F60915604809157040E945909CE01A5
:1024000001960E948A4C0431110514F00A501109FA
:10241000B80184EC93E00E948D318DEA93E00E9434
:10242000BE32882309F4A9CEA6CECF93DF9300D085
:1024300000D000D0CDB7DEB781E080936E0410925B
:10244000560486E08093570464EC71E0CE01019657
:102450000E94FC4CAE014F5F5F4F6091560480912B
:1024600057040E945909CE0101960E948A4C86E9C0
:1024700093E00E94D232882351F180915604811159
:1024800020C01092570464EC71E0CE0101960E94C6
:10249000FC4CAE014F5F5F4F609156048091570432
:1024A0000E945909CE0101960E948A4C10926E0436
:1024B00026960FB6F894DEBF0FBECDBFDF91CF9149
:1024C0000895853021F00E94A30A0E94B2108091E5
:1024D0005604853009F061C086E993E00E94133309
:1024E000882309F45AC064EC71E0CE0101960E9481
:1024F000FC4CAE014F5F5F4F609156048BE00E9431
:102500005909CE0101960E948A4C86E993E00E9407
:10251000E532882309F495C064EC71E0CE010196A0
:102520000E94FC4CAE014F5F5F4F6091560487E004
:102530000E945909CE0101960E948A4C80910A019D
:102540000E94C10864EC71E0CE0101960E94FC4C2F
:10255000AE014F5F5F4F60915604809157040E9417
:102560005909CE0101960E948A4C60ED77E080E027
:1025700090E00E94C74764EC71E0CE0101960E9492
:10258000FC4CAE014F5F5F4F6091560486E00E94A5
:102590005909CE0101960E948A4C8BED93E00E946E
:1025A000F9328823A9F01092560464EC71E0CE0150
:1025B00001960E94FC4CAE014F5F5F4F6091560444
:1025C000809157040E945909CE0101960E948A4CBD
:1025D0008DEA93E00E94D2328823F1F08091560474
:1025E0008F5F8093560490910A01891710F0109222
:1025F000560464EC71E0CE0101960E94FC4CAE01E1
:102600004F5F5F4F60915604809157040E945909B3
:10261000CE0101960E948A4C84EC93E00E94D23253
:10262000882309F424CF80915604811104C080913D
:102630000A01809356048091560481508093560479
:1026400003CF8BED93E00E94D232882309F45DCF53
:1026500092CF0F931F93CF93DF9300D000D000D081
:10266000CDB7DEB71092540461E771E0CE01019658
:102670000E94FC4CBE016F5F7F4F8FE594E00E948B
:10268000CC4E182FCE0101960E948A4C112319F0CE
:102690008FE08093540465E771E0CE0101960E94BB
:1026A000FC4CBE016F5F7F4F8FE594E00E94CC4EE3
:1026B000182FCE0101960E948A4C112319F08FE049
:1026C000809354046AE771E0CE0101960E94FC4CAD
:1026D000BE016F5F7F4F8FE594E00E94CC4E182FB4
:1026E000CE0101960E948A4C112319F081E180935A
:1026F00054046FE771E0CE0101960E94FC4CBE01CC
:102700006F5F7F4F8FE594E00E94CC4E182FCE0173
:1027100001960E948A4C112381F081E18093540438
:1027200013E0812F26960FB6F894DEBF0FBECDBF03
:10273000DF91CF911F910F91089564E871E0CE0170
:1027400001960E94FC4CBE016F5F7F4F8FE594E0C5
:102750000E94CC4E182FCE0101960E948A4C112364
:1027600019F083E18093540469E871E0CE01019689
:102770000E94FC4CBE016F5F7F4F8FE594E00E948A
:10278000CC4E182FCE0101960E948A4C112311F0D5
:1027900011E0C7CF6EE871E0CE0101960E94FC4CBB
:1027A000BE016F5F7F4F8FE594E00E94CC4E182FE3
:1027B000CE0101960E948A4C1111EACF63E971E0C3
:1027C000CE0101960E94FC4CBE016F5F7F4F8FE5EA
:1027D00094E00E94CC4E182FCE0101960E948A4CA4
:1027E0001111D6CF68E971E0CE0101960E94FC4C30
:1027F000BE016F5F7F4F8FE594E00E94CC4E182F93
:10280000CE0101960E948A4C1111C2CF6DE971E090
:10281000CE0101960E94FC4CBE016F5F7F4F8FE599
:1028200094E00E94CC4E182FCE0101960E948A4C53
:102830001111AECF62EA71E0CE0101960E94FC4C0C
:10284000BE016F5F7F4F8FE594E00E94CC4E182F42
:10285000CE0101960E948A4C11119ACF67EA71E06D
:10286000CE0101960E94FC4CBE016F5F7F4F8FE549
:1028700094E00E94CC4E182FCE0101960E948A4C03
:10288000111186CF6CEA71E0CE0101960E94FC4CDA
:10289000BE016F5F7F4F8FE594E00E94CC4E182FF2
:1028A000CE0101960E948A4C111172CF61EB71E04A
:1028B000CE0101960E94FC4CBE016F5F7F4F8FE5F9
:1028C00094E00E94CC4E182FCE0101960E948A4CB3
:1028D00011115ECF1091540411115ACF65EB71E0C4
:1028E000CE0101960E94FC4CBE016F5F7F4F8FE5C9
:1028F00094E00E94CC4E082FCE0101960E948A4C93
:10290000002311F012E00DCF6AEB71E0CE010196C9
:102910000E94FC4CBE016F5F7F4F8FE594E00E94E8
:10292000CC4E082FCE0101960E948A4C0111EACFAD
:102930006FEB71E0CE0101960E94FC4CBE016F5F0F
:102940007F4F8FE594E00E94CC4E082FCE01019678
:102950000E948A4C002309F4E4CED4CF1F93CF9376
:10296000DF93EC01BC0190E080E00E94390B182F4E
:102970002196BE0190E080E00E94390B612FDF912B
:10298000CF911F910C94864CEF92FF920F931F935F
:10299000CF93DF938C017B0164EC71E00E94FC4CCF
:1029A000D0E0C0E0B7016C0F7D1F90E080E00E9496
:1029B000390B682FC8010E946F4E2196CA30D1058D
:1029C00089F7C801DF91CF911F910F91FF90EF9090
:1029D00008954F925F926F927F928F929F92AF92E3
:1029E000BF92CF92DF92EF92FF920F931F93CF93FC
:1029F000DF93CDB7DEB72C970FB6F894DEBF0FBECE
:102A0000CDBF62EC71E088E797E00E94E54B2FE5CF
:102A100031E040E050E060E070E0CB010E945F0CEC
:102A200062EC71E088E797E00E94E54B1092550454
:102A3000D12CC12C80914F04909150048C159D0590
:102A400008F42CC1B60190E080E00E94390B7601B9
:102A50002FEFE21AF20A833109F01EC1B70190E0AC
:102A600080E00E94390B811117C1560182E0A80E47
:102A7000B11C712C612CC301B5010E94390B81116D
:102A80000BC1B6016C5F7F4FCE0107960E94C41444
:102A900065EC71E0CE0101960E94FC4CBE01695FBD
:102AA0007F4FCE0101960E94824E6BEC71E00E9436
:102AB000954EBC0188E797E00E94D34BCE0101966A
:102AC0000E948A4CCE0107960E948A4C00915504C0
:102AD00010E0000F111FF801EA50FD4FB182A082F3
:102AE000C6010E94AE14F801E254FD4F9183808329
:102AF00069EF71E088E797E00E94C14BB301A5013F
:102B0000CE0101960E941F0CBE016F5F7F4F88E7C8
:102B100097E00E94A04BCE0101960E948A4C66EE7F
:102B200071E088E797E00E94C14BC6010E94AE1495
:102B3000AC0170E060E0CE0101960E941F0CBE0166
:102B40006F5F7F4F88E797E00E94A04BCE01019610
:102B50000E948A4C65ED71E088E797E00E94C14BC6
:102B6000C6010E94AE148E0D9F1DAC0170E060E0A6
:102B7000CE0101960E941F0CBE016F5F7F4F88E758
:102B800097E00E94A04BCE0101960E948A4C64EC13
:102B900071E088E797E00E94C14B809155048F5FF8
:102BA0008093550464EA71E088E797E00E94C14B86
:102BB0000091550410E0460197E1890E911C000F29
:102BC000111FF801EA50FD4F91828082560125E1E4
:102BD000A20EB11CC5010E94AE14F801E254FD4FD3
:102BE00091838083A40170E060E0CE0101960E9491
:102BF0001F0CBE016F5F7F4F88E797E00E94A04BDC
:102C0000CE0101960E948A4C60E971E088E797E066
:102C10000E94C14BC5010E94AE148C0D9D1DAC01DC
:102C200070E060E0CE0101960E941F0CBE016F5F54
:102C30007F4F88E797E00E94A04BCE0101960E944B
:102C40008A4C62E871E088E797E00E94C14BC501B9
:102C50000E94AE1428E1C20ED11CC80ED91EA601D6
:102C600070E060E0CE0101960E941F0CBE016F5F14
:102C70007F4F88E797E00E94A04BCE0101960E940B
:102C80008A4C6FE671E088E797E00E94C14B809123
:102C900055048F5F809355046701CCCE66E571E0E3
:102CA00088E797E00E94C14B10E080915504181707
:102CB000C8F54AE050E0612F88E797E00E945C4C3D
:102CC000E12EF12CEE0CFF1CF701EA50FD4F408184
:102CD000518170E060E0CE0101960E941F0CBE01A0
:102CE0006F5F7F4F88E797E00E94D34BCE0101963C
:102CF0000E948A4CF701E254FD4F4081518170E0FF
:102D000060E0CE0101960E941F0CBE016F5F7F4FF5
:102D100088E797E00E94D34BCE0101960E948A4C2F
:102D20001F5FC3CF6BE371E088E797E00E947C4BA5
:102D30002C960FB6F894DEBF0FBECDBFDF91CF91BA
:102D40001F910F91FF90EF90DF90CF90BF90AF90C9
:102D50009F908F907F906F905F904F900895DF923B
:102D6000EF92FF920F931F93CF93DF93CDB7DEB710
:102D70006B970FB6F894DEBF0FBECDBF7C0110E09D
:102D800041E0B701CE0101960E943521DD24D394A4
:102D9000D10ECE0101960E947C1F082FCE01019614
:102DA0000E946A1F011112C0C7010E946A1F812F71
:102DB0006B960FB6F894DEBF0FBECDBFDF91CF91FB
:102DC0001F910F91FF90EF90DF9008951D2DD8CFA8
:102DD000DF92EF92FF920F931F93CF93DF93CDB7C4
:102DE000DEB76B970FB6F894DEBF0FBECDBF7C0188
:102DF000D62E10E041E0B701CE0101960E943521A8
:102E0000D11212C0CE0101960E940F1FBC018FE5A6
:102E100094E00E94FB4DCE0101960E94111F81118A
:102E200023C010926D0423C0CE0101960E947C1F26
:102E300001E0882339F31F5FCE0101960E946A1FCB
:102E40000111D8CFC7010E946A1F812F6B960FB660
:102E5000F894DEBF0FBECDBFDF91CF911F910F91D0
:102E6000FF90EF90DF90089581E080936D0400E083
:102E7000E2CFCF93DF93EC01FB01828193819B83AF
:102E80008A8384819581A681B7818C839D83AE835B
:102E9000BF8380859185A285B38588879987AA8716
:102EA000BB8789E192E0998388838DE03C96DE01BF
:102EB0001C9601900D928A95E1F7FB01818D928D10
:102EC0009A8F898FDF91CF9108950F931F93CF939E
:102ED000DF93CDB7DEB76B970FB6F894DEBF0FBEAA
:102EE000CDBF1092580409E514E0F80140815181EA
:102EF00021E060E774E0CE0101960E94BE20BE0191
:102F00006F5F7F4F82EF93E00E94060E62EF73E0E7
:102F1000CE0101960E943917CE0101960E94AF168C
:102F200080930B01F8014081518121E060E774E05A
:102F3000CE0101960E94BE20BE016F5F7F4F82EFDF
:102F400093E00E94060E1091580462EF73E0CE01E8
:102F500001960E943917612FCE0101960E94E81652
:102F60006B960FB6F894DEBF0FBECDBFDF91CF9149
:102F70001F910F9108950F931F93CF93DF93EC014F
:102F80008B0180916D04882341F060ED71E0C801F0
:102F90000E94604E81E080936D04B801CE010E94D2
:102FA000D24DCE01DF91CF911F910F9108950F93D4
:102FB0001F93CF93DF93CDB7DEB72C970FB6F8945E
:102FC000DEBF0FBECDBF0E94091060E083E00E940B
:102FD000134964ED71E088E797E00E94E54B05E650
:102FE00014E0F801108211826FE574E0CE010796BB
:102FF0000E94F24DBE01695F7F4FCE0101960E9493
:10300000BB17AE014F5F5F4F60E088E00E94590937
:10301000CE0101960E948A4CCE0107960E948A4CEE
:1030200060ED77E080E090E00E94C7476FE574E0D4
:10303000CE0107960E94F24DBE01695F7F4FCE011F
:1030400001960E94BB17AE014F5F5F4F60E0809119
:1030500057040E945909CE0101960E948A4CCE0164
:1030600007960E948A4C81E0F80182836FED71E03F
:10307000CE0101960E94FC4C6FE574E0CE010196F2
:103080000E94824EBC0188E797E00E94D34BCE019C
:1030900001960E948A4C2C960FB6F894DEBF0FBEA4
:1030A000CDBFDF91CF911F910F910895809145047D
:1030B00080934404809146048093450480914704A2
:1030C000809346048091480480934704809149048A
:1030D0008093480480914A0480934904809143047A
:1030E00081508093430420914F043091500421502B
:1030F00031093093500420934F04811108C068E1D6
:1031000072E088E797E00E947C4B0C94D7170895F3
:10311000CF93DF9380916904882369F0109269044A
:1031200080914D0490914E04009741F00197909347
:103130004E0480934D04DF91CF91089580916A04ED
:103140008823F1F140914B0450914C04D0914404F8
:1031500041155105C1F4D17080914504C82FCC1F91
:10316000CC27CC1F0E94561887E090E090934C0427
:1031700080934B04DC1709F181E080936B0481E0BC
:1031800080936C04D8CF8D2F90E09C01042E02C058
:10319000359527950A94E2F7D22FD1704150510905
:1031A000042E02C0959587950A94E2F7C82FC17046
:1031B00050934C0440934B04DDCF10926B04DFCF4F
:1031C00080916B048823D9F210926C04B4CF0F93D2
:1031D0001F93CF93DF9320916904222339F18B0150
:1031E000EC011092690480912E0390912F030097B7
:1031F00011F1029731F480913203909133030E94D0
:10320000121080912E0390912F03019731F4809139
:103210003003909131030E94121080912E039091FF
:103220002F03019790932F0380932E03DF91CF916B
:103230001F910F91089580916A048823B9F38091BA
:103240004B0490914C04892B41F40E94561888E05D
:1032500090E090934C0480934B0440914B04509128
:103260004C044150510950934C0440934B0420911D
:10327000440430E002C0359527954A95E2F7C8012D
:1032800020FFCE01DF91CF911F910F910C9412106E
:10329000E0915404F0E0EE0FFF1FE35FFB4F8081ED
:1032A00091810E9412108091290490912A04909398
:1032B0004E0480934D0410924204109241041092E7
:1032C000430488E090E090934C0480934B0481E0A9
:1032D00080936A0480936C040E940D100E948110F8
:1032E0000E94881880914F0490915004892BB1F767
:1032F0000C94D7179F92AF92BF92CF92DF92EF922A
:10330000FF920F931F93CF93DF93CDB7DEB72C9728
:103310000FB6F894DEBF0FBECDBF3FE7E32E39ED09
:10332000F32E48E0C42ED12C992493949091530409
:1033300080915504981708F077C06FE574E0CE01CE
:1033400007960E94F24DBE01695F7F4FCE01019644
:103350000E94BB17AE014F5F5F4F60E085E00E94A7
:103360005909CE0101960E948A4CCE0107960E940F
:103370008A4C00912504109126045801AA0CBB1C0C
:10338000809121049091220490933303809332031F
:10339000809123049091240490933103809330030F
:1033A000F0925204E092510480911D0490911E0409
:1033B00090932F0380932E038091530490E0880F05
:1033C000991FFC01EA50FD4F208131813093420466
:1033D0002093410482549D4FFC0180819181909300
:1033E000500480934F0410924304D0924C04C09236
:1033F0004B0410926A0490926C040E940D1080910C
:103400004F0490915004892B39F00E948110B5012E
:10341000C8010E94E718F3CF0E94D7178091530488
:103420008F5F8093530482CF2C960FB6F894DEBF43
:103430000FBECDBFDF91CF911F910F91FF90EF9005
:10344000DF90CF90BF90AF909F9008951F93CF9340
:10345000DF93CDB7DEB72C970FB6F894DEBF0FBE63
:10346000CDBF69E574E0CE0101960E94F24D6CEE8D
:1034700071E0CE0101960E94954E6FE574E00E94C6
:10348000824EBC01CE0107960E94F24DCE010196FC
:103490000E948A4C0E94291320912D0430912E0401
:1034A00011E0833019F5232B09F410E0BE01695FA8
:1034B0007F4FCE0101960E94F24D612FCE01019601
:1034C0000E94C20ECE0101960E948A4C0E944819A9
:1034D000CE0107960E948A4C2C960FB6F894DEBF58
:1034E0000FBECDBFDF91CF911F910895232B09F41B
:1034F00010E0BE01695F7F4FCE0101960E94F24D40
:10350000612FCE0101960E94370ECE0101960E94D6
:103510008A4C0E942913813011F40E9448190E949C
:1035200029138230A9F690E080E00E94E9140E94FD
:103530007A19CECF1F93CF93DF93CDB7DEB76B97BA
:103540000FB6F894DEBF0FBECDBF809158048F5FD9
:103550008093580490910B01891710F01092580431
:103560004091590450915A0421E060E774E0CE0183
:1035700001960E94BE20BE016F5F7F4F82EF93E0F5
:103580000E94060E1091580462EF73E0CE0101967E
:103590000E943917612FCE0101960E94E8166B96A2
:1035A0000FB6F894DEBF0FBECDBFDF91CF911F9154
:1035B00008951F93CF93DF93CDB7DEB76B970FB608
:1035C000F894DEBF0FBECDBF80915804811104C0B6
:1035D00080910B018093580480915804815080930E
:1035E00058044091590450915A0421E060E774E076
:1035F000CE0101960E94BE20BE016F5F7F4F82EF19
:1036000093E00E94060E1091580462EF73E0CE0121
:1036100001960E943917612FCE0101960E94E8168B
:103620006B960FB6F894DEBF0FBECDBFDF91CF9182
:103630001F910895CF93DF9300D000D000D0CDB775
:10364000DEB780916D04882301F16CEE71E0CE014C
:1036500001960E94FC4C6FE574E0CE0101960E9439
:10366000824EBC0189E594E00E94594ECE0101963C
:103670000E948A4C0E94651726960FB6F894DEBF0A
:103680000FBECDBFDF91CF9108950E94261AF4CFCF
:10369000CF93DF9300D000D000D0CDB7DEB764EC7D
:1036A00071E089E594E00E94AF4E882359F00E94B2
:1036B000151226960FB6F894DEBF0FBECDBFDF9170
:1036C000CF9108956CEE71E0CE0101960E94FC4C02
:1036D000BE016F5F7F4F89E594E00E943A4FBC01C5
:1036E00089E594E00E94754FCE0101960E948A4CB4
:1036F0000E946517DECF0F931F93CF93DF93CDB753
:10370000DEB7A1970FB6F894DEBF0FBECDBF0E9403
:10371000031080910A010E94F90861E08CE00E9488
:10372000D74860911504709116048CE00E942E48D1
:1037300061E083E00E94D74860E083E00E94134983
:1037400062E08FE00E94D74820E042E060E188E339
:1037500093E00E947A4626E040E052EC61E070E09F
:1037600088E797E00E94514A41E060E088E393E0F7
:103770000E9461466EEE71E088E393E00E94AE4BDA
:1037800001E021E04CE362E086E593E00E944D41D8
:10379000811106C061E271E088E797E00E94C14BA9
:1037A00010926D0381E090E0909369038093680329
:1037B000909367038093660386E593E00E942F4110
:1037C00061E086E593E00E94D23E0AE010E01093AB
:1037D00063030093620386E090E090936503809317
:1037E000640366E171E086E593E00E94C14B1093AB
:1037F00063030093620386E190E0909365038093F6
:1038000064036BE071E086E593E00E94C14B86E5BE
:1038100093E00E94C4446CE271E080E090E00E947A
:10382000C7476FEE70E088E797E00E94C14B67EDF5
:1038300070E088E797E00E94C14B64EF71E080E0A0
:1038400090E00E94C74765E080E794E00E94A21FD5
:10385000811129C06CE271E080E090E00E94C747CE
:1038600080E00E944149892BF1F46BEB70E088E71E
:1038700097E00E94C14B6FEF71E0CE0101960E946C
:10388000FC4CAE014F5F5F4F60915604809157042E
:103890000E945909CE0101960E948A4C6CED75E098
:1038A00080E090E0CECF68EA70E088E797E00E9481
:1038B000C14B6CE870E088E797E00E94C14B0E9422
:1038C0002D090E94840D21E044EC51E060E774E092
:1038D000CE0101960E94BE20BE016F5F7F4F82EF36
:1038E00093E00E94060E62EF73E0CE0101960E9403
:1038F0003917CE0101960E94AF1680930B014AE062
:1039000050E0682F88E797E00E945C4C21E044EC8F
:1039100051E060E774E0CE0101960E94BE20BE0136
:103920006F5F7F4F82EF93E00E94060E1091580464
:1039300062EF73E0CE0101960E943917612FCE012C
:1039400001960E94E8166FE574E0CE014C960E9445
:10395000F24DBE01645E7F4FCE0101960E94BB17FF
:10396000BE016F5F7F4F88E797E00E94D34BCE0187
:1039700001960E948A4CCE014C960E948A4C10926D
:1039800057046FE574E0CE014C960E94F24DBE01E3
:10399000645E7F4FCE0101960E94BB17AE014F5F60
:1039A0005F4F60E0809157040E945909CE01019653
:1039B0000E948A4CCE014C960E948A4C0AEA20E072
:1039C00030E640E050E060E070E0CB010E94CB0BBD
:1039D000A1960FB6F894DEBF0FBECDBFDF91CF9199
:1039E0001F910F910895CF93DF93CDB7DEB72C973A
:1039F0000FB6F894DEBF0FBECDBF8DEA93E00E94F4
:103A0000D232882309F49AC00E949A1A6FE574E0B2
:103A1000CE0107960E94F24DBE01695F7F4FCE0135
:103A200001960E94BB17AE014F5F5F4F60E080912F
:103A300057040E945909CE0101960E948A4CCE017A
:103A400007960E948A4C84EC93E00E94D23288232D
:103A500009F47CC00E94D91A6FE574E0CE01079684
:103A60000E94F24DBE01695F7F4FCE0101960E9418
:103A7000BB17AE014F5F5F4F60E0809157040E941B
:103A80005909CE0101960E948A4CCE0107960E94E8
:103A90008A4C86E993E00E94D232882309F45EC002
:103AA0000E941A1B6FE574E0CE0107960E94F24D4A
:103AB000BE01695F7F4FCE0101960E94BB17AE0128
:103AC0004F5F5F4F60E0809157040E945909CE011B
:103AD00001960E948A4CCE0107960E948A4C8BED7B
:103AE00093E00E94D232882309F440C00E94481B10
:103AF0006FE574E0CE0107960E94F24DBE01695F4A
:103B00007F4FCE0101960E94BB17AE014F5F5F4F02
:103B100060E0809157040E945909CE0101960E94ED
:103B20008A4CCE0107960E948A4C2C960FB6F894C8
:103B3000DEBF0FBECDBFDF91CF91089560E08DEA6B
:103B400093E00E942D3381115FCF7DCF60E084EC44
:103B500093E00E942D3381117DCF9BCF60E086E9F9
:103B600093E00E942D3381119BCFB9CF60E08BEDA4
:103B700093E00E942D338111B9CFD7CF8F929F92BE
:103B8000AF92BF92CF92DF92EF92FF920F9364ECCD
:103B900071E08FE594E00E94FC4C64EC71E089E5F3
:103BA00094E00E94FC4C82EF93E00E94FC1E20E017
:103BB00040E06DE28BED93E00E94B93120E040E0FF
:103BC0006EE284EC93E00E94B93120E040E06FE2C5
:103BD0008DEA93E00E94B93120E040E060E386E99D
:103BE00093E00E94B93180EA882E86E8982EAA24B4
:103BF000A394B12C90E8C92E9AE1D92E96E0E92E33
:103C0000F12C0FEF29EC36E040E260E886E593E026
:103C10000E94953F6AE072E080E593E00E94FC4CD0
:103C200029E1C22E38E1E32E07E126E145E164E116
:103C300088E393E00E9416470F91FF90EF90DF908A
:103C4000CF90BF90AF909F908F90089580E593E0C4
:103C50000E948A4C86E593E00E94E03F89E594E06B
:103C60000E948A4C8FE594E00C948A4CCF93DF93AA
:103C70001F92CDB7DEB76983DC01ED91FC91028024
:103C8000F381E02D41E050E0BE016F5F7F4F099569
:103C90000F90DF91CF910895DC0159968D919C9101
:103CA000009739F0DC01ED91FC910480F581E02D65
:103CB000099490E080E00895CF93DF93EC01E98DC3
:103CC000FA8D309749F481E090E09B838A8390E0FD
:103CD00080E0DF91CF91089513821282898D9A8DB1
:103CE0000E94152BE98DFA8D22813381232B59F700
:103CF000F0CFFC01818D928D009719F061E00C945A
:103D000045280895CF93DF931F92CDB7DEB741E0EA
:103D100050E0BE016F5F7F4F0E943526019731F45E
:103D2000898190E00F90DF91CF9108958FEF9FEF01
:103D3000F9CFFC01818D928D009711F00C94821EB9
:103D40008FEF9FEF08950F931F93CF93DF93EC01B5
:103D5000898D9A8D10E000E0009799F00E94821EF4
:103D60008C010F3F100769F0898D9A8DFC01428507
:103D700053856485758541505109610971090E9417
:103D8000B127C801DF91CF911F910F910895EF9254
:103D9000FF920F931F93CF93DF93EC017B018A0176
:103DA0001B821A8288EE93E0A0E0B0E08C839D83B2
:103DB000AE83BF8389E192E0998388838DE190E0AF
:103DC0000E94D34F9A8F898F009779F02DE1F701E8
:103DD000DC0101900D922A95E1F74CE050E0B8012A
:103DE000CE010C960E942652188EDF91CF911F9122
:103DF0000F91FF90EF900895FC011382128288EEDC
:103E000093E0A0E0B0E084839583A683B78389E143
:103E100092E091838083128E118E148608950C9601
:103E20000895DC015996ED91FC91309721F081E0E5
:103E30009581923008F480E00895DC015996ED9167
:103E4000FC91309729F06285738584859585089566
:103E50006FEF7FEFCB010895DC015996ED91FC9156
:103E6000309729F06389748985899689089560E07F
:103E700070E0CB010895CF92DF92EF92FF92CF9343
:103E8000DF93FC01218D328D232B09F1EC010E947F
:103E90002C1F6B017C01CE010E941D1FA701960102
:103EA000261B370B480B590BDA01C901811530E885
:103EB0009307A105B10520F08FEF9FE7A0E0B0E0E8
:103EC000DF91CF91FF90EF90DF90CF90089590E039
:103ED00080E0F6CFCF93DF93EC01898D9A8D009728
:103EE00041F00E949A28898D9A8D0E946F501A8EF7
:103EF000198EDF91CF910895DC015996ED91FC91D7
:103F0000309721F081E09581911101C080E0089502
:103F10000F931F93CF93DF93EC018B0141E00E943D
:103F20006930811109C040E0B801CE01DF91CF9125
:103F30001F910F910C94693081E0DF91CF911F9117
:103F40000F9108950F931F93CF93DF93EC01162FDA
:103F50008FA5882321F0CE018A960E949A28412FAE
:103F600061E0CE010E94BA22811102C090E011C02E
:103F70008E01045F1F4FBE01C8010E94881F882365
:103F8000A9F3B801CE018A960E94E52591E0882325
:103F900069F3892FDF91CF911F910F910895FC0153
:103FA000DB0112968D919C911397938382838BE210
:103FB00092E09183808314968C9114978483159654
:103FC0008C911597858316964D915D916D917C919D
:103FD000199746835783608771871A964D915D9133
:103FE0006D917C911D9742875387648775871E96D4
:103FF0004D915D916D917C91519746875787608B6C
:10400000718B52968C915297828B53964D915D9104
:104010006D917C915697438B548B658B768B57961D
:104020004D915D916D917C915A97478B508F618F27
:10403000728F5B968D919C91948F838F08954F9290
:104040005F926F927F928F929F92AF92BF92CF9228
:10405000DF92EF92FF920F931F93CF93DF93CDB731
:10406000DEB7C754D1090FB6F894DEBF0FBECDBF7F
:104070005C014A01390119A218A28BE292E09F8FDC
:104080008E8F1BA21C821B829A8389831E82645F8F
:104090007F4F7E018EE1E80EF11CC7010E94E525ED
:1040A0008401FE0131966F015E2C4F2C6FE270E0AF
:1040B000C8010E940B52009709F455C0F8012081F5
:1040C0002F3219F40F5F1F4FF1CF801B8D3008F096
:1040D0008CE0E82EF12CA701B801CE01CB960E940E
:1040E0002652EBE3F0E0EC0FFD1FEE0DFF1D1082FA
:1040F000C6010E949A2821E0AE01455C5F4F652D04
:10410000742DC6010E94272A811121C0F501138256
:1041100012828BE292E0918380831582C501C95B94
:10412000DF4F0FB6F894DEBF0FBECDBFDF91CF914A
:104130001F910F91FF90EF90DF90CF90BF90AF90C5
:104140009F908F907F906F905F904F9008950E0D8D
:104150001F1D852D942D0E949A28C2015C2C4D2C88
:10416000C92ED82EA3CF08191909F3011183008392
:10417000652D742DC5010E94CF1FD0CFCF92DF9245
:10418000FF920F931F93CF93DF93CDB7DEB7C9553F
:10419000D1090FB6F894DEBF0FBECDBF6C018A0106
:1041A000F22E9E01285A3F4FCE01CB960E941F202F
:1041B0006A968EAD9FAD6A97080F191FF80180812E
:1041C000811110C0BE01655C7F4FCE0101960E9437
:1041D000CF1F4CEE51E0BE016F5F7F4FC6010E94C2
:1041E000C71E0FC019A218A28BE292E09F8F8E8F7C
:1041F0001BA221968FAD2197811113C0C6010E9489
:10420000FC1EC601C75ADF4F0FB6F894DEBF0FBEC3
:10421000CDBFDF91CF911F910F91FF90DF90CF9095
:1042200008952F2DA801BE01655C7F4FCE014E96EB
:104230000E94272A882311F3CE01CB960E949A2848
:104240008F2D8670863041F449A95AA96BA97CA9A3
:10425000CE014E960E94B127BE01625E7F4FCE0115
:1042600001960E94CF1FA801B6CFDF92EF92FF9276
:104270000F931F93CF93DF93CDB7DEB7C756D10906
:104280000FB6F894DEBF0FBECDBF8C017B01D42EDC
:10429000BE016F5F7F4FF701818D928D0E943C2799
:1042A00018161CF48981811104C0C8010E94FC1EEB
:1042B00036C0853E69F38E3259F38C8583FDE8CF95
:1042C00022961FAE1EAE22978BE292E09FAF8EAF7A
:1042D00024961FAE2497BE01655A7F4FCE010196EA
:1042E0000E948725F701618D728D2D2DAE01455AF3
:1042F0005F4FCE01CE960E94272A8823B1F2BE01DD
:10430000625C7F4FCE0181960E94CF1FAE01455A5D
:104310005F4FBE016F5D7F4FC8010E94C71EC8017D
:10432000C959DF4F0FB6F894DEBF0FBECDBFDF9186
:10433000CF911F910F91FF90EF90DF900895E0E7EC
:10434000F4E0158216821186138682E090E0A0E0E8
:10435000B0E084879587A687B78713A215A614A611
:104360008BE292E093A782A717A608959FB7F894CF
:104370002091C7068091C506213019F489BF9FBFDF
:1043800008958FBF08952091C706222381F03FB77B
:10439000F8942091C706213069F429B72093C50607
:1043A00049B72091C6062095242329BF3FBF8DB968
:1043B0009EB908953093C506FACF8FEF0C94530938
:1043C00061E0FC0184810E9413498091B904882333
:1043D00039F01092B9048091C70681110C94B6216E
:1043E0000895CF93DF93EC018091B904811109C046
:1043F00081E08093B9048091BA049091BB040E943B
:10440000C32160E08C81DF91CF910C941349CF934D
:10441000DF93EC018E81882389F08F8198859C0140
:104420002F5F3F4F38872F838230924018F40E94CD
:10443000DD21F3CFCE010E94E0211E82DF91CF91DA
:104440000895673030F026E1FC01258360E0862F77
:104450000895623011F130F4662389F06130B9F0CB
:1044600083E508C06430D9F081E5643018F082E556
:104470006530B1F78093BA041092BB0406C080E5A2
:104480008093BA0481E08093BB0461E0E0CF80E5D3
:104490008093BA041092BB04DACF81E5F1CF82E5B4
:1044A000EFCF0F931F93CF93DF93EB010E949547BC
:1044B0008B010E94DD218F3F69F00E949547601BB0
:1044C000710B6C177D07A8F380E0DF91CF911F91EE
:1044D0000F91089581E0F9CF8F929F92AF92BF9292
:1044E000FF920F931F93CF93DF93EC01F62E4901B8
:1044F0005A010E940722CE010E94F1216CE271E074
:10450000CE010E9451228F2D80640E94530908E140
:1045100010E0D501C401002E04C0B695A79597956B
:1045200087950A94D2F70E94530908501109083F51
:104530008FEF180771F785E9FF2021F088E0F81266
:104540000DC087E80E94530910E00E94DD218A8790
:1045500087FF06C01F3F21F01F5FF7CF8FEFF2CF1D
:10456000DF91CF911F910F91FF90BF90AF909F90DF
:104570008F9008958F929F92AF92BF92EF92FF9289
:104580000F931F93CF93DF93EC01E62E1B861986C2
:104590001E821D824C830E9495478B0161E08C81B5
:1045A0000E94D74861E08C810E9413490E946B33BE
:1045B00082E58093BA041092BB048091BA04909172
:1045C000BB040E94C3212AE0F22E8FEF0E94530900
:1045D000FA94F110FACF8091C70681110E94B6219A
:1045E000CE010E94F12120E030E0A90160E0CE017F
:1045F0000E946C22F82E8A8781E0F816C1F00E9492
:104600009547601B710B613D774068F381E08D83B6
:10461000CE010E94E02180E0DF91CF911F910F91A8
:10462000FF90EF90BF90AF909F908F9008952AEAEF
:1046300031E040E050E068E0CE010E946C2282FF51
:1046400025C0FB868B85812C912C5401823029F466
:10465000812C912CA12C80E4B82E20E030E0A9011F
:1046600067E3CE010E946C22A501940169E2CE01AC
:104670000E946C228A878823C1F00E949547601BA4
:10468000710B613D774048F388E0C1CF94E0F92E8B
:104690000E94DD218A87FA94F110FACF8A3A11F04C
:1046A00082E0B5CF82E08B87CDCF8B858230C1F49D
:1046B00020E030E0A9016AE3CE010E946C22882349
:1046C00011F086E0A4CF0E94DD21807C803C11F4B3
:1046D00083E08B870E94DD210E94DD210E94DD2185
:1046E000CE010E94E0216E2DCE01DF91CF911F916E
:1046F0000F91FF90EF90BF90AF909F908F900C9490
:1047000021220F931F93CF93DF93EC010E949547D3
:104710008B010E94DD218A878F3F91F40E9495478B
:10472000601B710B6D327140A0F38FE08D83CE0161
:104730000E94E02180E0DF91CF911F910F910895B9
:104740008E3F11F08DE0F2CF81E0F5CFCF92DF9276
:10475000EF92FF920F931F93CF93DF93EC016901C8
:10476000C801820F931F8130924048F58E818823C3
:1047700071F088819981AA81BB8184179507A6076A
:10478000B70729F48F819885C816D90670F5488334
:1047900059836A837B838B85833039F089E0440FAA
:1047A000551F661F771F8A95D1F79A01AB0161E10A
:1047B000CE010E946C22882379F083E08D83CE01A4
:1047C0000E94E02180E0DF91CF911F910F91FF9037
:1047D000EF90DF90CF900895CE010E94812388232F
:1047E00071F318861F8281E08E838F8198858C15E6
:1047F0009D0560F06701E00EF11EEC14FD0471F000
:104800000E94DD21F60181936F01F7CF0E94DD2127
:104810008F819885019698878F83E7CF8F819885C0
:10482000080F191F18870F838985882319F0011530
:10483000124018F0CE010E94072281E0C4CFEF920F
:10484000FF920F931F930115110539F00E94A623C3
:104850001F910F91FF90EF90089581E0F9CFEF92B3
:10486000FF920F931F93790100E012E030E020E007
:104870000E94A6231F910F91FF90EF900895EF9251
:10488000FF920F931F93CF93DF938C01862F7A01B2
:104890000E945309E7018EEFF81A89910E9453098B
:1048A000CE15DF05D1F78FEF0E9453098FEF0E94DD
:1048B00053090E94DD21F80182878F71853069F0EC
:1048C00081E18583C8010E94E02180E0DF91CF91E2
:1048D0001F910F91FF90EF90089581E0F7CFEF9235
:1048E000FF920F93CF93DF93EC01790182E14115A1
:1048F00051056105710599F08B85833039F089E0A8
:10490000440F551F661F771F8A95D1F79A01AB0197
:1049100068E1CE010E946C22882339F084E08D8307
:10492000CE010E94E02180E025C0A7016EEFCE01FC
:104930000E943F248823A1F30023C1F068E572E0C0
:10494000CE010E945122811102C085E1E8CF20E012
:1049500030E0A9016DE0CE010E946C22882311F0A5
:1049600084E1DDCF0E94DD218111FACFCE010E94CA
:10497000E02181E0DF91CF910F91FF90EF900895BA
:104980001F93CF93DF93EC010E94F1210E94DD2160
:10499000182FCE010E94E02181E01F3F09F480E042
:1049A000DF91CF911F910895EAEBF4E080E58083D9
:1049B00011820895CF93DF93EC019C012A5F3F4F52
:1049C00041E050E060E070E08B8D9C8D0E94082FEC
:1049D0008823B9F08F89988DA98DBA8D892B8A2B60
:1049E0008B2B59F48C814E815F81688579854F8B43
:1049F000588F698F7A8F80688C838C8180628C83DA
:104A000081E0DF91CF9108958F929F92AF92BF92F4
:104A1000CF92DF92EF92FF92CF93DF93EC010E944F
:104A2000DA2481110CC080E0DF91CF91FF90EF90EC
:104A3000DF90CF90BF90AF909F908F900895EB8DB7
:104A4000FC8DCE80DF80E884F98482E0C81AD1082A
:104A5000E108F108858504C0CC0CDD1CEE1CFF1CB0
:104A60008A95D2F786859785A089B189C80ED91E07
:104A7000EA1EFB1E848146015701880E911CA11C71
:104A8000B11C8C149D04AE04BF0461F081E0881A4F
:104A90009108A108B108C501B4010E94552D8111EA
:104AA000F0CFC1CFEB8DFC8D258580E092E0A0E0BA
:104AB000B0E004C0880F991FAA1FBB1F2A95D2F728
:104AC0004B895C896D897E89840F951FA61FB71F4E
:104AD0008B8B9C8BAD8BBE8B81E0A6CFCF93DF936E
:104AE000EC01462F6E857F85888999890E94192D52
:104AF000882351F08A8920E2829FC00111248B53C0
:104B00009B4FDF91CF91089590E080E0FACFCF9353
:104B1000DF93DC0190E0E0E08EE22D91203291F015
:104B2000983029F4EB01CE0FD11D8883EF5FAB01E4
:104B30004E0F511D9D0121503109E9012881EA01E3
:104B40002883EF5F9F5F9B3041F7E60FF72FF11D42
:104B50001082DF91CF910895FB019B01255F3F4FAC
:104B600040E241932E173F07E1F7DC0120E037E0F8
:104B70009D91492F992319F19E3229F43A3059F029
:104B800028E03AE0F5CFECE8F5E08491882329F0BD
:104B900031969813FACF80E017C03217A8F05FED76
:104BA000590F5E3588F48FE9890F8A3110F440EE91
:104BB000490FFB01E20FF11D40832F5FD9CF81E048
:104BC000FB019081903239F308950F931F93CF9397
:104BD000DF93FC012581222331F080E0DF91CF912A
:104BE0001F910F9108958B01EC01FB0187898031A2
:104BF00039F582E08D831F8A188E198E1A8E808D6A
:104C0000918DB0E0A0E025E0880F991FAA1FBB1F7F
:104C10002A95D1F78B8B9C8BAD8BBE8B1C8F0B8F0A
:104C200081E08C831E821F82188619861A861B8655
:104C30001C861D861E861F86188A198A1A8ACECF60
:104C4000803259F683E08D83428D538D648D758D4E
:104C50004F8B588F698F7A8F9E012D5E3F4FC80111
:104C60000E94FB2D8111DACFB8CF2F923F924F9245
:104C70005F926F927F928F929F92AF92BF92CF92EC
:104C8000DF92EF92FF920F931F93CF93DF93EC018C
:104C90005B012A018D81811115C08FEF9FEFDF919C
:104CA000CF911F910F91FF90EF90DF90CF90BF9029
:104CB000AF909F908F907F906F905F904F903F90BC
:104CC0002F9008958C8180FFE8CF0B891C892D8956
:104CD0003E894A855B856C857D85C201B0E0A0E098
:104CE00068017901C41AD50AE60AF70AC816D90676
:104CF000EA06FB0618F42801441A550A42011E016F
:104D000026E0220E311C8114910409F4B3C04A85B7
:104D10005B856C857D856A0181E0D8228B8D9C8DB9
:104D20008A019B01E9E03695279517950795EA9545
:104D3000D1F7ED81E230E1F5FC01628D738D848D58
:104D4000958D600F711F821F931F612C22E0722EC0
:104D50006C187D088614970408F434012C8126FD14
:104D600004C06114F2E07F0671F400910C0110910F
:104D70000D0120910E0130910F010617170728072A
:104D8000390709F053C040E00E94192D882309F427
:104D900084CFC6018B539B4FD5019C01260D371D37
:104DA000FC012E173F0709F460C041914D93F9CFE4
:104DB000FC0174807A947022C114D10471F47110D2
:104DC0000CC0452B462B472B39F58F89988DA98D23
:104DD000BA8D8E839F83A887B987EB8DFC8D6E81FA
:104DE0007F8188859985625071098109910925859E
:104DF00004C0660F771F881F991F2A95D2F7068572
:104E0000178520893189600F711F821F931F670DDD
:104E1000711D811D911D99CF4E815F8168857985B6
:104E200091010E947A2D8111D8CF37CF750183016E
:104E30009601AB01BC018091C3049091C4040E940F
:104E40001F24882309F429CFA60CB71C8A859B85CB
:104E5000AC85BD85860D971DA11DB11D8A879B87D9
:104E6000AC87BD87861897084ECF281B390BA20E3A
:104E7000B31EECCFC20113CF0F931F93CF93DF93D9
:104E8000FC012581223040F1EB018C018285938564
:104E9000A485B5858F719927AA27BB27892B8A2BD3
:104EA0008B2BD1F440E250E0BE01C8010E943526B0
:104EB000803279F49881992389F0953E99F39E3256
:104EC00089F39B8593FDEECFDF91CF911F910F91D9
:104ED0000895880F880BF8CF8FEFF6CF80E0F4CFDE
:104EE000FF920F931F93CF93DF931F92CDB7DEB73F
:104EF000FC0125812230C8F08C01428553856485F0
:104F0000758585E076956795579547958A95D1F78C
:104F1000F42FFF70FF2E41E050E0BE016F5F7F4F26
:104F2000C8010E943526019719F090E080E012C078
:104F3000F80182859385A485B5854F96A11DB11D85
:104F400082879387A487B587F0E2FF9EC001112472
:104F50008B539B4F0F90DF91CF911F910F91FF903B
:104F600008958F929F92AF92BF92CF92DF92EF926D
:104F7000FF920F931F93CF93DF93EC018D818111EB
:104F80000EC080E0DF91CF911F910F91FF90EF90C5
:104F9000DF90CF90BF90AF909F908F9008950B8936
:104FA0001C892D893E89041715072607370748F302
:104FB0004A015B01823031F48A869B86AC86BD86CD
:104FC00081E0E0CF81149104A104B10449F41E8270
:104FD0001F82188619861A861B861C861D86F0CFAE
:104FE0000A851B852C853D85EB8DFC8D858590E0A4
:104FF0000996B901A8014150510961097109082EAA
:1050000004C076956795579547950A94D2F7750130
:105010006401E1E0CE1AD108E108F10804C0F69479
:10502000E794D794C7948A95D2F7C416D506E606B6
:10503000F70620F0012B022B032B11F58F89988D99
:10504000A98DBA8D8E839F83A887B9878E010A5F49
:105050001F4FC114D104E104F10409F4ADCF4E8116
:105060005F816885798598018B8D9C8D0E947A2D52
:1050700091E0C91AD108E108F1088111EACF81CF86
:10508000C41AD50AE60AF70AE1CFFF920F931F93DD
:10509000CF93DF93FC012581222309F444C0F62E2F
:1050A000EC01848187FF32C061E0CF010E946E2550
:1050B0008C01892BC1F18D81823048F48B899C89C8
:1050C000AD89BE89F801848F958FA68FB78F8F89A0
:1050D000988DF801938F828F8F89988DA98DBA8DC5
:1050E000B58BA48BE091BC04F091BD04309759F0CE
:1050F000B8016A5E7F4FC80148960995F801808D16
:10510000918D938B828B8C818F778C83F11003C070
:105110008C818F7E8C838F2DDF91CF911F910F918A
:10512000FF900C94EF2C80E0DF91CF911F910F91B5
:10513000FF900895CF93DF93EC0161E00E94452832
:10514000882311F01D8281E0DF91CF910895CF93E4
:10515000DF93EC018D81813029F090E080E0DF91D8
:10516000CF9108958C8181FFF8CF82FD13C080918B
:10517000C3049091C4040E94C0248111EECF8C819D
:1051800085FF1BC060E0CE010E9445288C818F7D89
:105190008C83E3CF4B895C896D897E898A859B8569
:1051A000AC85BD8584179507A607B70701F3CE0127
:1051B0000E94B1278111DBCFD0CF4091BE04509126
:1051C000BF046091C0047091C104452B462B472B4E
:1051D00021F080E00E94CB2CC0CF80618C832A8597
:1051E0003B85317080E092E0821B930BB8CF4F92E9
:1051F0005F926F927F928F929F92AF92BF92EF9247
:10520000FF920F931F93CF93DF9300D000D0CDB7C1
:10521000DEB7FC0185818130A1F080E00F900F9016
:105220000F900F90DF91CF911F910F91FF90EF9012
:10523000BF90AF909F908F907F906F905F904F90B6
:105240000895848181FFE9CF83899489A589B689EE
:1052500084179507A607B70700F3892B8A2B8B2B9A
:1052600009F478C04A015B017F014284538464845D
:105270007584CF010E94B127882379F2F701838DCD
:10528000948D81149104A104B10451F54789508D86
:10529000618D728D0E941330882309F4BECFF7010F
:1052A000178A108E118E128EF701838A948AA58A2E
:1052B000B68A84818068848361E0C7010E944528A2
:1052C000882309F4AACFB501A40144165506660641
:1052D000770610F4B301A201C7010E94B1279ECF47
:1052E00046815781608571859E012F5F3F4F0E94E7
:1052F0007A2D882309F491CFF701838D948D49810C
:105300005A816B817C81FC0127892031F1F408EFFF
:105310001FEF20E030E0401751076207730720F6C7
:105320000E941330882309F478CFF7014681578112
:10533000608571850FEF1FEF2FEF3FE0838D948D18
:105340000E94662E8111B0CF68CF08EF1FEF2FEFBC
:105350003FE0E1CF81E062CFCF92DF92EF92FF9208
:105360001F93CF93DF93EC0180E2689FF00111243B
:10537000EB53FB4F9385917161F0842F827449F058
:1053800080E0DF91CF911F91FF90EF90DF90CF9061
:105390000895142F6A8B80910C0190910D01A091BA
:1053A0000E01B0910F018E879F87A88BB98BC4889F
:1053B000D588F12CE12C7601DD24CC24CF8AD88E3F
:1053C000E98EFA8E828D938DB0E0A0E0AC01BD0134
:1053D0004C295D296E297F294F8B588F698F7A8FD1
:1053E0008385887129F5848D958DA68DB78D8B8BDE
:1053F0009C8BAD8BBE8B81E08D83812F8F708C83D6
:105400001E821F82188619861A861B861C861D8698
:1054100081E016FFB6CF40E050E0BA01CE01DF9147
:10542000CF911F91FF90EF90DF90CF900C94F728D1
:10543000803109F0A5CF9E012D5E3F4F8B8D9C8D55
:105440000E94FB2D882309F49BCF84E0D5CFBF9227
:10545000CF92DF92EF92FF920F931F93CF93DF9340
:10546000CDB7DEB72B970FB6F894DEBF0FBECDBF1A
:10547000FC01358131110BC0C22E8B017C01BE01B4
:105480006F5F7F4FCA010E94AC25811102C080E08E
:10549000A2C0F801838D948DF701948F838FF8015A
:1054A0001682178210861186128613861486158638
:1054B000B12CF80182859385A485B58543895489EB
:1054C0006589768984179507A607B70788F525E0CB
:1054D000B695A795979587952A95D1F7F82FFF70E0
:1054E000DF2EC8010E947027009789F2FC012081FD
:1054F000222341F0253E09F05AC0BB2029F0BB24ED
:10550000B394D7CFB1100EC0F701D28A40910C01ED
:1055100050910D0160910E0170910F0146875787E0
:10552000608B718BFC0180818111E9CFBB24B39426
:105530008C2D8271823109F0AACFBB2009F45BC0A7
:1055400061E0C7010E946E258C01892B09F49FCF71
:1055500080E2F80111928A95E9F78BE0FE0131961D
:10556000D80101900D928A95E1F7E091BC04F09189
:10557000BD04309709F44FC0B801625F7F4FC80186
:1055800040960995F80180899189938B828B918F40
:10559000808F86859785978B868B81E00E94EF2C84
:1055A000882309F474CF4C2DF701628911C04BE0B8
:1055B00050E0BC01CE0101960E94EE51892B09F00A
:1055C00078CF8C2D80734C2D6D2D803309F45FCFF7
:1055D000C7010E94AC292B960FB6F894DEBF0FBE10
:1055E000CDBFDF91CF911F910F91FF90EF90DF9092
:1055F000CF90BF900895F8018581823009F447CF9C
:10560000C8010E940425882309F441CFF701128ABA
:1056100005EC14E09DCF81E298E2F801918B808B3C
:1056200080E098E097878687ADCF2F923F924F9288
:105630005F926F927F928F929F92AF92BF92CF9222
:10564000DF92EF92FF920F931F93CF93DF9300D0DF
:1056500000D01F92CDB7DEB77C016B011A01DC01CF
:1056600015968C911597813009F0CAC014961C913B
:1056700011FFC6C012FDB0C0410112951F701095F8
:1056800011701D83D7011A960D911D912D913C919A
:105690001D978114910409F426C15B968D919C910C
:1056A0005C97FC0174807A94B901A80129E0769591
:1056B0006795579547952A95D1F774221170711007
:1056C00020C001151105E9F416964D915D916D917B
:1056D0007C911997411551056105710509F099C033
:1056E00057968D919D910D90BC91A02D0097A1058D
:1056F000B10509F0B0C0C7010E94DA24882309F47B
:105700007FC080E092E0801B910B540188159905C1
:1057100008F45C01D7015B964D915C915C971696FD
:105720008D919D910D90BC91A02D0297A109B10979
:10573000FA01258504C0880F991FAA1FBB1F2A954F
:10574000D2F74685578560897189840F951FA61FFA
:10575000B71F9C01AD01270D311D411D511D2901B0
:105760003A01A11432E0B30609F07BC080910C012C
:1057700090910D01A0910E01B0910F018415950536
:10578000A605B70559F48FEF9FEFDC0180930C015C
:1057900090930D01A0930E01B0930F010D8196011E
:1057A000B301A2018091C3049091C4040E946F24AC
:1057B000882331F19EEFD91A8A189B08F701828558
:1057C0009385A485B5858A0D9B1DA11DB11D82877A
:1057D0009387A487B58756CFF70143895489658994
:1057E000768982859385A485B585481759076A0708
:1057F0007B0709F441CFC7010E94B12781113CCF3B
:1058000081E090E0D70113969C938E93129780E0ED
:1058100007C09E012F5F3F4F0E947A2D811102C069
:1058200090E07BC089819A81AB81BC81F701238D97
:10583000348DF901278948EF5FEF60E070E0203197
:1058400021F048EF5FEF6FEF7FE084179507A60721
:10585000B70708F050CFF70186839783A087B187F9
:1058600050CF0115110591F5D7011A964D915D9113
:105870006D917C911D9753968D919D910D90BC914A
:10588000A02D481759076A077B0700F181E00E94A5
:10589000EF2C882309F4B4CF40920C0150920D01F3
:1058A00060920E0170920F018091C204816080931A
:1058B000C2040B531B4FD601C8018A0D9B1DF80172
:1058C0008E179F0759F02D912193FACF41E0C30124
:1058D000B2010E94192D8111ECCF92CF801B910B48
:1058E000C80ED91E69CF14968C91149753964D917A
:1058F0005D916D917C915697401751076207730730
:1059000020F5F701038B148B258B368B80688483FD
:10591000F701848183FD26C0C1010F900F900F9085
:105920000F900F90DF91CF911F910F91FF90EF900B
:10593000DF90CF90BF90AF909F908F907F906F90AF
:105940005F904F903F902F9008952091BC0430912C
:10595000BD04232BE9F221143104D1F2806814969E
:105960008C93D6CF61E0C7010E944528882309F4B3
:1059700047CFD2CFCF93DF931F92CDB7DEB76983E6
:1059800041E050E0BE016F5F7F4F0E94152B0F90EA
:10599000DF91CF9108950F934091BE045091BF04C1
:1059A0006091C0047091C1044115510561057105F4
:1059B00099F0082F25EC34E08091C3049091C40441
:1059C0000E946F24882349F01092BE041092BF04F5
:1059D0001092C0041092C10481E00F9108950F93BA
:1059E000CF939091C204911102C081E015C0C82FDD
:1059F00040910C0150910D0160910E0170910F01C9
:105A0000082F25EC34E08091C3049091C4040E94D7
:105A10006F24811104C080E0CF910F910895CC23B1
:105A200021F38C2F0E94CB2C8823A9F31092C2045F
:105A3000DCCFCF92DF92EF92FF92CF936B017C018C
:105A4000C42F80910C0190910D01A0910E01B09195
:105A50000F018C159D05AE05BF0501F181E00E9487
:105A6000EF2C811107C080E0CF91FF90EF90DF9085
:105A7000CF90089525EC34E0B701A6018091C304CE
:105A80009091C4040E942F24882369F3C0920C01D2
:105A9000D0920D01E0920E01F0920F014091C204EC
:105AA0004C2B4093C20481E0DFCFCF92DF92EF9284
:105AB000FF926B017C0181E00E94EF2C8823A9F00A
:105AC000E5ECF4E0119286E0E53CF807D9F7C092E6
:105AD0000C01D0920D01E0920E01F0920F01809125
:105AE000C20481608093C20481E0FF90EF90DF9058
:105AF000CF9008958F929F92AF92BF92CF92DF92F4
:105B0000EF92FF920F931F93CF93DF93FC01818558
:105B10009285A385B4850196A11DB11D84179507B3
:105B2000A607B70770F480E0DF91CF911F910F9126
:105B3000FF90EF90DF90CF90BF90AF909F908F90AD
:105B4000089583889488A588B6888789803189F5E7
:105B5000BB27A72F962F852FE9016A017B018F01B3
:105B6000BC01CD01680D791D8A1D9B1D80900C0123
:105B700090900D01A0900E01B0900F01861697062F
:105B8000A806B90601F5F8018789803111F5DD24F1
:105B9000EE24FF24F601EE0FFF1FEB53FB4F808135
:105BA0009181B0E0A0E088839983AA83BB8381E0E0
:105BB000BBCFDB01CA01C7E0B695A795979587953E
:105BC000CA95D1F7C9CF40E00E94192D8111DBCFD2
:105BD000AACFE894C7F8DD24EE24FF24F601EE0FE7
:105BE000FF1FEE0FFF1FEB53FB4F80819181A281BE
:105BF000B381BF70D8CF4F925F926F927F92AF9276
:105C0000BF92CF92DF92EF92FF920F931F93CF93A9
:105C1000DF9300D000D0CDB7DEB78C0149835A8323
:105C20006B837C835901C12CD12C7601412C82E0FD
:105C3000582E612C712C49815A816B817C819E0187
:105C40002F5F3F4FC8010E947A2D882339F1F80158
:105C50008585A301920104C0220F331F441F551FE5
:105C60008A95D2F7DA01C901C80ED91EEA1EFB1EB9
:105C700049815A816B817C818789803111F188EF5C
:105C80009FEFAFEFBFE0481759076A077B0798F20D
:105C9000F501C082D182E282F38281E00F900F9001
:105CA0000F900F90DF91CF911F910F91FF90EF9088
:105CB000DF90CF90BF90AF907F906F905F904F90AC
:105CC000089588EF9FEFA0E0B0E0DDCF4F925F92A4
:105CD0006F927F928F929F92AF92BF92CF92DF92FC
:105CE000EF92FF920F931F93CF93DF93EC0142301B
:105CF00051056105710590F480E0DF91CF911F910E
:105D00000F91FF90EF90DF90CF90BF90AF909F905A
:105D10008F907F906F905F904F90089589859A85BE
:105D2000AB85BC850196A11DB11D84179507A607FB
:105D3000B70710F3CB88DC88ED88FE888F89803127
:105D400009F042C0BB27A72F962F852F4801590184
:105D50002A013B01C80ED91EEA1EFB1E80910C01D0
:105D600090910D01A0910E01B0910F01C816D906B6
:105D7000EA06FB0699F58F898031C1F5B301A201CE
:105D8000552766277727440F551F4B535B4FFA0162
:105D9000918280828091C20481608093C2048A894A
:105DA000823080F08D819E81AF81B8858C0D9D1DE4
:105DB000AE1DBF1D8093BE049093BF04A093C0048A
:105DC000B093C10481E099CFDB01CA01E7E0B69549
:105DD000A79597958795EA95D1F7B8CF40E0C70189
:105DE000B6010E94192D8111C6CF86CFB301A20141
:105DF0004F77552766277727440F551F440F551FA8
:105E00004B535B4FFA0180829182A282B382C2CF50
:105E10002F923F924F925F926F927F928F929F92BA
:105E2000AF92BF92CF92DF92EF92FF920F931F93A8
:105E3000CF93DF93CDB7DEB72F970FB6F894DEBFC1
:105E40000FBECDBF3C01488759876A877B873F8358
:105E50002E83D901CD90DD90ED90FC90C114D1043A
:105E6000E104F10439F0BFEFCB1ADB0AEB0AFB0ABD
:105E70001D8210C0FC01C080D180E280F380F1E07F
:105E8000FD83088519852A853B850130110521058B
:105E9000310571F7F30181859285A385B4858C0165
:105EA0009D010F5F1F4F2F4F3F4F0C871D872E8780
:105EB0003F8746015701212C312C2101F3018185B7
:105EC0009285A385B485281639064A065B0608F034
:105ED00044C00C851D852E853F85081519052A05AA
:105EE0003B0550F482E0882E912CA12CB12C92E03D
:105EF000C92ED12CE12CF12C9E012F5F3F4FB50113
:105F0000A401C3010E947A2D882339F1D501C4016F
:105F10000196A11DB11D49815A816B817C81452B60
:105F2000462B472BA9F5AC01BD014C195D096E0943
:105F30007F09088519852A853B8540175107620727
:105F4000730741F50FEF1FEF2FEF3FE0B501A401FD
:105F5000C3010E94662E811125C01D828D812F965E
:105F60000FB6F894DEBF0FBECDBFDF91CF911F916A
:105F70000F91FF90EF90DF90CF90BF90AF909F90E8
:105F80008F907F906F905F904F903F902F900895EB
:105F90006C017D011FEF211A310A410A510A4C019F
:105FA0005D018CCFC814D904EA04FB0488F4140101
:105FB000250121E0221A3108410851089501840188
:105FC000B201A101C3010E94662E52014101C3CF5B
:105FD000AE81BF814D915D916D917C9141155105CF
:105FE0006105710561F4EE81FF81C082D182E28298
:105FF000F382FD81F1110BC001E00D83AFCF97015A
:106000008601C3010E94662E8111EDCFA6CF1FEF3E
:10601000C11AD10AE10AF10AD301CD92DD92ED92C3
:10602000FC9213979BCFAF92BF92CF92DF92EF92E9
:10603000FF920F931F93CF93DF9300D000D0CDB783
:10604000DEB75C016A017B0182E090E0A0E0B0E095
:10605000F50180839183A283B3839E012F5F3F4F1D
:10606000B701A601C5010E947A2D882381F100E0C5
:1060700010E09801B701A601C5010E94662E882391
:1060800031F1C980DA80EB80FC80F50187898031AD
:10609000C9F088EF9FEFAFEFBFE0C816D906EA0658
:1060A000FB06D8F281E00F900F900F900F90DF91D8
:1060B000CF911F910F91FF90EF90DF90CF90BF9005
:1060C000AF90089588EF9FEFA0E0B0E0E6CF80E0CA
:1060D000EACF8F929F92AF92BF92CF92DF92EF92D0
:1060E000FF920F931F93CF93DF93EC01142F7093C4
:1060F000C4046093C304442309F478C0453070F0AD
:1061000080E0DF91CF911F910F91FF90EF90DF9092
:10611000CF90BF90AF909F908F90089540E060E047
:1061200070E0CB010E94192D882351F3812F8150FB
:10613000990BAC0164E0440F551F6A95E1F74B538E
:106140005B4FFA01E254FE4F80818F77C9F63C968F
:1061500080819181A281B38184369105A105B10529
:1061600078F24A535E4FFA01C080D180E280F3801A
:10617000C114D104E104F10419F240E0C701B601F1
:106180000E94192D882309F4BBCF8091D0049091EF
:10619000D1048115924009F0B3CF9091D504992391
:1061A00009F4AECF2091D3043091D404232B09F409
:1061B000A7CF8091D204882309F4A2CF9A8B8C8335
:1061C0001D8690E041E050E02D85E22FBA01022EBD
:1061D00002C0660F771F0A94E2F78617970751F0FF
:1061E00031E0320F3D87283078F38ACFC12CD12C93
:1061F0007601C3CF2091DB043091DC0450E040E015
:106200002115310541F42091E9043091EA044091CF
:10621000EB045091EC042D833E834F83588780918B
:10622000D3049091D40446015701880E991EA11CF5
:10623000B11C8B8A9C8AAD8ABE8A0091D6041091CB
:10624000D704198F088FA091D504B0E00E94C84FE1
:10625000DC01CB01880D991DAA1DBB1D8A8F9B8F68
:10626000AC8FBD8F25E0000F111F2A95E1F701507B
:106270001E4F012F11270695800F911FA11DB11DE3
:106280008E879F87A88BB98B0091D8041091D90471
:1062900030E020E00115110541F40091E504109172
:1062A000E6042091E7043091E804C81AD90AEA0A02
:1062B000FB0AC00ED11EE21EF31E04C0F694E79442
:1062C000D794C794EA95D2F7C986DA86EB86FC861E
:1062D0008CE025EFC2162FE0D206E104F10440F075
:1062E00085EFC8168FEFD806E104F10420F480E1B1
:1062F0008F8B81E006CF8091F1049091F204A09100
:10630000F304B091F4048A8F9B8FAC8FBD8F80E231
:10631000EFCFFC01768365830895FC017287618766
:106320000895CF93DF93EC01898160FB83F9898322
:1063300085FD1AC08A816623D1F060E00E94D748AB
:106340008A8190E0FC01E353F04FE491F0E0EE0F1E
:10635000FF1FEE5FFF4E259134913D8B2C8BFC018E
:10636000E856F04FE491EE8BDF91CF91089562E013
:10637000E5CF1F93CF93DF93EC01122F1A822CE30A
:1063800030E03C832B8324EF31E03E832D8338873C
:106390002F8320E931E03A8729871B861C861D86DA
:1063A0001E861F86188A198A1A8A1B8A89816F3F5E
:1063B00081F06A838F7D8983642FCE010E949131A1
:1063C00089818B7E10FB81F98983DF91CF911F91A9
:1063D00008958062F0CFFC01218160FB24F92183C4
:1063E00008958F929F92AF92BF92CF92DF92EF92D9
:1063F000FF920F931F93CF93DF93EC01898182FD6E
:1064000014C085FD12C0EC89FD8920813E8981FB85
:10641000992790F983FB882780F98927922F932366
:1064200021E009F020E082278A8B0E949547AB018A
:10643000BC019A892B898881992309F47BC0211199
:1064400079C080FD5DC0816088834E875F87688BDF
:10645000798B8B89882319F1992309F10D811E818C
:1064600030E020E0CE84DF84E888F9884A015B01CF
:106470008C189D08AE08BF0875016401C016D106CE
:10648000E206F30660F0888181FD09C02B852D8727
:106490008A648F7788834E875F87688B798B0E85B8
:1064A0001F8528893989401B510B620B730B0F81A3
:1064B000188530E020E0401751076207730750F05D
:1064C0008B85882339F0911105C08C871B868881C4
:1064D00084608883898186FF06C01C8698819B7FA3
:1064E00098838F7B8983DF91CF911F910F91FF90CC
:1064F000EF90DF90CF90BF90AF909F908F900895D6
:106500000E851F85288939896A017B01C01AD10A45
:10651000E20AF30A0B811C8130E020E0C016D106AC
:10652000E206F30608F4BBCF21E02B8B8062806883
:1065300088838FCF8E7F888391118BCF222309F49C
:10654000AECF1B8A81FD03C08B858F5F8B878881CF
:106550008D7F806188834E875F87688B798B86FF0C
:1065600004C01C861B868F7B8883888187FF97CF1A
:106570008F7788838981816089836BCFCF93DF9305
:10658000EC01898184FF03C0CE010E94F131988122
:1065900094FB882780F994FF02C09F7E9883DF9147
:1065A000CF910895CF93DF93EC01898184FF03C0DD
:1065B000CE010E94F1319981892F817090FF02C034
:1065C0009E7F9983DF91CF910895CF93DF93EC0164
:1065D000898184FF03C0CE010E94F131988193FB31
:1065E000882780F993FF02C0977F9883DF91CF912E
:1065F0000895CF93DF93EC01898184FF03C0CE011E
:106600000E94F131988192FB882780F992FF06C0A1
:106610009C85923031F4998190649983DF91CF9178
:10662000089580E0FBCFCF93DF93EC01898184FF55
:1066300003C0CE010E94F131988192FB882780F936
:1066400092FF06C09C85933031F4998190649983C0
:10665000DF91CF91089580E0FBCFCF92DF92EF9250
:10666000FF921F93CF93DF93EC01162F898184FF54
:1066700003C0CE010E94F1318B85811751F010E0EB
:10668000812FDF91CF911F91FF90EF90DF90CF90FE
:106690000895888186FB112710F986FFF0CF0E94AC
:1066A0009547CE84DF84E888F988AB01BC014C199A
:1066B0005D096E097F0989859A85B0E0A0E04817D9
:1066C00059076A077B07D8F20E9495476E877F8734
:1066D000888B998BD5CFCF93CFB7F8948091C8068C
:1066E000811123C0E5EDFFE08491E0EAFFE09491A1
:1066F000E82FF0E0EE0FFF1FEE5DFF4EA591B49185
:10670000EC91E92321F461E088E00E94134961E003
:1067100088E00E94D7486C9A6E9A61E089E00E94F6
:10672000D74861E08AE00E94D7488091C8068F5F11
:106730008093C806CFBFCF9108958091FD069091B8
:10674000FE06891B990B08959091FE068091FD0627
:106750002FEF3FEF981748F4E92FF0E0E150F94FA1
:10676000208130E09F5F9093FE06C9010895E0917B
:10677000FE068091FD06E81730F4F0E0E150F94F95
:10678000808190E008958FEF9FEF08950895CF9353
:10679000DF93EC01E091D506F091D6063097F1F049
:1067A0009091FE068091FD069817C0F090E0292F89
:1067B00030E02617370754F4DE01A20FB31F4C91C7
:1067C0002150394FD9014C939F5FF1CF1092FE06B3
:1067D0006093FD06CB01DF91CF910994DF91CF91BA
:1067E0000895E091D706F091D806309729F01092DD
:1067F000DB061092DA0609940895CF93DF931F9277
:10680000CDB7DEB769832091D9062223F9F0209114
:10681000DA06203258F021E030E0FC013383228395
:1068200090E080E00F90DF91CF9108958091DB069A
:10683000E82FF0E0E452F94F998190838F5F8093C5
:10684000DB068093DA0681E090E0ECCF61E0CE01D8
:1068500001960E942035F7CFCF92DF92EF92FF9200
:106860000F931F93CF93DF937C01CB018A0120917B
:10687000D906222389F0EB016B01C40ED51ECC157D
:10688000DD0569F06991D701ED91FC910190F081EE
:10689000E02DC7010995F3CF642F0E942035C80170
:1068A000DF91CF911F910F91FF90EF90DF90CF90EC
:1068B00008951092FE061092FD061092DB061092CB
:1068C000DA060E94A23481EF93E30E944C3587ECF4
:1068D00093E30C944735CB01BA010C94BD3481E0AD
:1068E0008093D9066093FC061092DB061092DA06BC
:1068F00008950C946F340F93062F21E04091DA062F
:106900006CED76E08091FC060E94D0341092DB069C
:106910001092DA061092D9060F91089561E00C9456
:106920007B34E9ECF6E01382128288EE93E0A0E07B
:10693000B0E084839583A683B78387E392E0918355
:106940008083089510926E0781E080936C07109207
:106950006B0761E083E10E94134961E082E10E94DC
:106960001349E1E7F0E080818C7F808388E48093A5
:10697000700085E48093740008959B01AC0160E091
:1069800074E284EF90E00E948E4F2051310941095A
:10699000510956954795379527952093700008958E
:1069A0000F93413208F044C090916E079111FCCFD3
:1069B00092E090936E0700936C079FEF90931F07F0
:1069C00070936607609365071092640740936307AE
:1069D00010926D0790916D07880F892B80936D073A
:1069E00080916B07813011F510926B0780916D07D4
:1069F000809373008091740083FDF8CF85EC8093C1
:106A00007400222321F080916E078230D1F38091AF
:106A10001F078F3F79F080911F07803269F08091C6
:106A20001F07803359F084E00F91089585EEE7CF7A
:106A300081E0FACF80E0F8CF82E0F6CF83E0F4CFB8
:106A400020914107260F3327331F21323105ECF403
:106A500020916E07FC0190E080E0243069F082E034
:106A60000895A09141072191AC014D5B584FA40FAF
:106A7000B52FB11D2C930196861798F3809141078D
:106A8000680F6093410780E0089581E00895909336
:106A9000680780936707089590936A078093690752
:106AA000089585ED809374008091740084FDFCCF7F
:106AB00010926E07089585EC8093740010926E0713
:106AC00008951F920F920FB60F9211240BB60F92DA
:106AD0002F933F934F935F936F937F938F939F93E6
:106AE000AF93BF93EF93FF9380917100887F8036BF
:106AF00009F44EC008F041C0883209F4AAC028F554
:106B0000803109F49EC0C8F4882309F407C1883095
:106B100009F497C0FF91EF91BF91AF919F918F9131
:106B20007F916F915F914F913F912F910F900BBE8D
:106B30000F900FBE0F901F901895883109F489C0EF
:106B4000803241F780931F0715C0803409F4A6C036
:106B500048F48033B9F38833E9F680931F070E9425
:106B60005B35D8CF803509F489C0883509F49EC0DB
:106B7000883481F60E945135CDCF883909F494C00C
:106B800038F5883729F050F4883611F0803711F63F
:106B900083E080936E071092200757C0883809F46D
:106BA00083C0803919F0803809F0B4CF8091200774
:106BB000803208F079C0E091200781E08E0F809349
:106BC000200780917300F0E0EF5DF84F80833DC0B7
:106BD000803B39F0E0F4803A09F485C0883A09F046
:106BE00099CF84E080936E0710924207109241077C
:106BF000E0916907F0916A07099580914107811139
:106C00000FC081E0809341071092430709C0803C88
:106C100009F482C0883C09F47FC0883B09F07ACF30
:106C2000E091420781E08E0F80934207F0E0ED5B38
:106C3000F84F8081809373009091420780914107C3
:106C400031C080916D078093730085EC8093740050
:106C500061CF90916407809163079817B8F5809190
:106C6000650790916607E091640721E02E0F20935D
:106C70006407E80FF92FF11D8081E5CF20916507AA
:106C800030916607E091640781E08E0F809364077E
:106C900080917300E20FF32FF11D808390916407C0
:106CA00080916307981788F285E8D0CF2091650717
:106CB00030916607E091640781E08E0F809364074E
:106CC00080917300E20FF32FF11D808380916C0798
:106CD000811150CF81E080936B0784EA8093740028
:106CE00010926E0717CF0E945B358091200780328B
:106CF00030F4E0912007F0E0EF5DF84F10826091F2
:106D0000200770E0E0916707F091680781E297E063
:106D1000099510922007FECE85ECE0CF10921F0758
:106D200029CF2F923F924F925F926F927F928F92D4
:106D30009F92AF92BF92CF92DF92EF92FF920F930A
:106D40001F93CF93DF9300D000D000D0CDB7DEB734
:106D50003C016A013E832D83FC82EB825801A41A18
:106D6000B50AB7FE03C0B194A194B1088D809E808E
:106D7000861A970A97FE03C09194819491088A1409
:106D80009B045CF0902F812F0D811E819D838E834B
:106D90009C2D8D2D6B01692F782F0C151D055CF036
:106DA0009D818E817E836D83692F782F902F812F17
:106DB0008601C92ED82E1601201A310A2B012D81E9
:106DC0003E81421A530A57FE03C051944194510820
:106DD000710137FE03C03FEFE31AF30AF594E7941D
:106DE0008D819E81861797075CF5A1E0B0E0BA839C
:106DF000A983C016D1064CF1D301ED91FC91048416
:106E0000F585E02D2B813C81A8016D817E818A145E
:106E10009B041CF04D815E81B801C3010995E41803
:106E2000F508F7FE0AC02D813E8189819A81280FDD
:106E3000391F3E832D83E20CF31C0F5F1F4FD9CF08
:106E40002FEF3FEF3A832983D4CF26960FB6F894DD
:106E5000DEBF0FBECDBFDF91CF911F910F91FF908D
:106E6000EF90DF90CF90BF90AF909F908F907F90EA
:106E70006F905F904F903F902F9008950895DC01A0
:106E8000ED91FC910084F185E02D09940F931F93FF
:106E9000DC01ED91FC91048CF58DE02D09951F919D
:106EA0000F9108950F931F93DC01ED91FC91068CD7
:106EB000F78DE02D09951F910F910895EF92FF92A4
:106EC0000F931F93DC01ED91FC9100A0F1A1E02D47
:106ED00009951F910F91FF90EF9008958F929F92C7
:106EE000AF92BF92CF92DF92EF92FF920F931F93D8
:106EF000CF93DF93EC015B014A0169017801E881DE
:106F0000F9810284F385E02D0995C80CD91C86010E
:106F100001501109E881F9810488F589E02D950176
:106F2000A401B501CE010995E881F9810688F789A8
:106F3000E02DCE01DF91CF911F910F91FF90EF9047
:106F4000DF90CF90BF90AF909F908F9009948F92D9
:106F50009F92AF92BF92CF92DF92EF92FF920F93E8
:106F60001F93CF93DF93EC015B014A016901E88134
:106F7000F9810284F385E02D099595012C0D3D1DC5
:106F800021503109E881F9810488F589E02D7801E3
:106F90008401A401B501CE010995E881F981068833
:106FA000F789E02DCE01DF91CF911F910F91FF90D6
:106FB000EF90DF90CF90BF90AF909F908F9009940B
:106FC0004F925F926F927F928F929F92AF92BF92F9
:106FD000CF92DF92EF92FF920F931F93CF93DF93A5
:106FE0006C012B015A0139014801DC01ED91FC9142
:106FF0000284F385E02D0995E201640C751CD6012D
:10700000ED91FC91C615D7055CF40088F189E02D5F
:1070100087019401A501BE01C60109952196EFCF14
:107020000688F789E02DC601DF91CF911F910F915E
:10703000FF90EF90DF90CF90BF90AF909F908F9098
:107040007F906F905F904F900994EF92FF920F9313
:107050001F93DC011A960D911C911B9718962D9188
:107060003C911997ED91FC9100A0F1A1E02D7B01DD
:1070700050E040E070E060E009951F910F91FF90B3
:10708000EF9008956F927F928F929F92AF92BF92EE
:10709000CF92DF92EF92FF920F931F93CF93DF93E4
:1070A000EC016B015A0139014801E881F981028440
:1070B000F385E02D0995E881F9810288F389E02DB7
:1070C00087019301A501B601CE010995A501480DDF
:1070D000591D41505109E881F9810288F389E02D59
:1070E0009301B601CE010995E881F9810088F18903
:1070F000E02D9401A501B601CE010995C60CD71C5F
:10710000B60161507109E881F9810088F189E02DAB
:107110009401A501CE010995E881F9810688F789D6
:10712000E02DCE01DF91CF911F910F91FF90EF9055
:10713000DF90CF90BF90AF909F908F907F906F9097
:10714000099408956F927F928F929F92AF92BF920F
:10715000CF92DF92EF92FF920F931F93CF93DF9323
:107160005C01EB016A01490138018701DC01ED9105
:10717000FC916217730719F5641675062CF0962DAD
:10718000872D3A01C92ED82E9601261937092F5F6F
:107190003F4F048CF58DE02DA301BE01C50109957B
:1071A000DF91CF911F910F91FF90EF90DF90CF90E3
:1071B000BF90AF909F908F907F906F9008954615ED
:1071C000570591F42617370724F0892D4B01C22F5C
:1071D000D82F9E01281939092F5F3F4F068CF78D54
:1071E000E02DA601B401DACF0284F385E02D0995E4
:1071F000D501ED91FC910488F589E02D830194017E
:10720000A601BE01C5010995D501ED91FC91068845
:10721000F789E02DC501DF91CF911F910F91FF906C
:10722000EF90DF90CF90BF90AF909F908F907F9026
:107230006F900994FC016370668B8481958126812F
:107240003781613039F0633029F091878087338747
:107250002287089531872087938782870895FC01CC
:107260001382128289E492E0918380837583648320
:10727000578346837187608753874287168A1586AE
:1072800014861786168681E0858B848B2FEF3FEF5F
:10729000338B228B318B208B878B108E128E118E2D
:1072A00008952F923F924F925F926F927F928F92AA
:1072B0009F92AF92BF92CF92DF92EF92FF920F9385
:1072C0001F93CF93DF9300D000D000D0CDB7DEB7AF
:1072D0009E838D834B013A016901802F21E030E0CC
:1072E00029014C185D08222433242C183D08220C57
:1072F000331CB12CA12C01E010E0982F94709983DD
:10730000A82FA270AA83B82FB870BB8381708C831A
:10731000AC14BD040CF0A7C057FC08C081E0C81A2B
:10732000D10892E0290E311C420C531CAFEFAA1A6F
:10733000BA0A0E5F1F4F400E511EB981BB2311F1D7
:10734000AD81BE81ED91FC9111970484F585E02D0E
:107350009701A601460D571DB4016A0D7B1DCD0195
:107360000995AD81BE81ED91FC9111970484F5855D
:10737000E02D9701A3014A0D5B1DB601680D791D33
:10738000CD010995BA81BB2311F1AD81BE81ED918B
:10739000FC9111970484F585E02D9701A3014C1908
:1073A0005D09B4016A0D7B1DCD010995AD81BE81DA
:1073B000ED91FC9111970484F585E02D9701A301CF
:1073C0004A195B09B601680D791DCD010995BB818C
:1073D000BB2311F1AD81BE81ED91FC911197048425
:1073E000F585E02D9701A3014A0D5B1DB4016C19D1
:1073F0007D09CD010995AD81BE81ED91FC9111977B
:107400000484F585E02D9701A601460D571DB401B2
:107410006A197B09CD010995BC81BB2309F478CF9A
:10742000AD81BE81ED91FC9111970484F585E02D2D
:107430009701A3014A195B09B4016C197D09CD01BB
:107440000995AD81BE81ED91FC9111970484F5857C
:10745000E02D9701A3014C195D09B4016A197B095C
:10746000CD01099555CF26960FB6F894DEBF0FBE15
:10747000CDBFDF91CF911F910F91FF90EF90DF90E3
:10748000CF90BF90AF909F908F907F906F905F90C4
:107490004F903F902F9008952F923F924F925F927E
:1074A0006F927F928F929F92AF92BF92CF92DF9214
:1074B000EF92FF920F931F93CF93DF93CDB7DEB779
:1074C00028970FB6F894DEBF0FBECDBF5C017A835C
:1074D00069832A0149013801201731070CF0BFC028
:1074E0003C832B83C90137FDBFC0AB81BC81B595FF
:1074F000A795BC83AB838B819C8198878F83E8168B
:10750000F90614F4F886EF82D501ED91FC9102841E
:10751000F385E02DC50109958F819885880F991F06
:107520009C838B837401E81AF90A29803A80AF8121
:10753000B8852A0E3B1ED501ED91FC910288F38996
:10754000E02D86019701A201B101C5010995C30192
:10755000840D951D9E838D83AC0141505109D50149
:10756000ED91FC910288F389E02D9701B101C501ED
:1075700009958B819C81681A790AAF81B8854A0E7A
:107580005B1ED501ED91FC910088F189E02D9301FE
:10759000A20169817A81C501099589819A81880E44
:1075A000991EB40161507109D501ED91FC910088DB
:1075B000F189E02D9301A201C5010995760101E051
:1075C0002F813885A201B101C5010E9451398F81F7
:1075D0009885881A990A91E0891A910802E02F810A
:1075E0003885A201B401C5010E9451396D807E80A9
:1075F000AF81B8856A1A7B0AB1E06B1A710804E0A2
:107600002F813885A301B401C5010E94513908E0DA
:107610002F813885A301B101C5010E945139D501DF
:10762000ED91FC910688F789E02DC50128960FB6EB
:10763000F894DEBF0FBECDBFDF91CF911F910F91A8
:10764000FF90EF90DF90CF90BF90AF909F908F9082
:107650007F906F905F904F903F902F9009941C8384
:107660000B8317FF42CFC80101969C838B833DCFCC
:107670003F924F925F926F927F928F929F92AF92C2
:10768000BF92CF92DF92EF92FF920F931F93CF930F
:10769000DF93CDB7DEB72A970FB6F894DEBF0FBEE3
:1076A000CDBF9A8789877E836D8358874F83290151
:1076B0003701DC01ED91FC910284F385E02D099501
:1076C000C801079697FD07969C0193E0359527958D
:1076D0009A95E1F73A832983912C812CB12CA12C26
:1076E000312C8F8198858A0D9B1D9C838B83A614DA
:1076F000B704ACF5F12CE12CE016F10644F5C70116
:1077000087709927330C892B59F4F70183E0F5959D
:10771000E7958A95E1F7E80DF91DE40DF51D349024
:1077200037FE11C0A985BA85ED91FC9111970484AB
:10773000F585E02D96014B815C816D817E816E0D1A
:107740007F1DCD010995BFEFEB1AFB0AD5CF2FEFB7
:10775000A21AB20A89819A81880E991EC2CFA98580
:10776000BA85ED91FC9111970688F789E02DCD013E
:107770002A960FB6F894DEBF0FBECDBFDF91CF9132
:107780001F910F91FF90EF90DF90CF90BF90AF903F
:107790009F908F907F906F905F904F903F90099453
:1077A0002F923F924F925F926F927F928F929F9211
:1077B000AF92BF92CF92DF92EF92FF920F931F93FF
:1077C000CF93DF93CDB7DEB76A970FB6F894DEBFDD
:1077D0000FBECDBF9A8F898F7A8369834A01D22EDB
:1077E00018870F833701BC2CDC0159962D913C91F1
:1077F0005A972115310509F015C118968D919C9164
:107800001997681779070CF0D7C11A968D919C913A
:10781000481759070CF0D0C14C2C512CB6E0CB9E28
:10782000600D711D11247C876B87161617060CF0EE
:10783000C3C1EA2DF0E0FA87E98793E0EE0FFF1F5E
:107840009A95E1F7F88BEF87CF01840F951F1816F3
:1078500019060CF0B1C1A98DBA8D58968C91811181
:1078600004C0BFEABD1508F4D394A98DBA8DED917B
:10787000FC9111970284F385E02DCD010995B5E0C7
:10788000DB9EC0011124E981FA81FC83EB83312C5A
:10789000212C9C0124563A4F388F2F8B4A2D50E0D3
:1078A0005E8B4D8BEF89F88DE20DF31D44919E8226
:1078B0008D82D12CC12C69817A81620D731D7A8BE6
:1078C000698B842F90E09C8B8B8BE98DFA8DA08146
:1078D000B18140FF82C0F1E0BF126FC0AF126DC036
:1078E0001C96ED91FC912F813885A4014C0D5D1DF6
:1078F00069897A89898D9A8D0995EB89FC89F59535
:10790000E7954E2F5FEFC51AD50A6D817E818D896F
:107910009E89680F791F7E836D8398E0C916D10414
:1079200081F6AFEF2A1A3A0AEB81FC81E40DF51DCE
:10793000FC83EB83F5E02F16310409F0B3CF2F81E0
:10794000388526153705B9F0A98DBA8DED91FC91D2
:10795000B1E0BB1257C0AB1255C069817A816B5F31
:107960007F4F0088F189E02D830128E030E0A401F9
:10797000898D9A8D0995A98DBA8DED91FC911197FC
:107980000688F789E02DCD016A960FB6F894DEBF20
:107990000FBECDBFDF91CF911F910F91FF90EF9060
:1079A000DF90CF90BF90AF909F908F907F906F901F
:1079B0005F904F903F902F9009941E96ED91FC910F
:1079C000EF80F88409851A8592014D815E816B8173
:1079D0007C81898D9A8D099590CF2F8138852615C8
:1079E000370509F48ACF31E0B31207C0A31205C0EE
:1079F0001C96ED91FC91930178CF1E96ED91FC9130
:107A00007301E0CF6B857C85641975090684F78561
:107A1000E02D73010F8518899201A401898D9A8D3B
:107A20000995A9CFF90134969491329745915491D3
:107A3000D91AB7E0DB9E400D511D1124F9012591A3
:107A400034913C8B2B8BFA0125903490FA013296BD
:107A5000749031963491398B32966490319644907B
:107A600041E04C1518F04A1508F07FC0662D062C31
:107A7000000C770B7C836B83842D042C000C990BFA
:107A80009E838D83A98DBA8DED91FC91119702840F
:107A9000F385E02DCD010995512CD12CC12CEA2D77
:107AA000F0E0FA87E9872B2D30E03C872B87A40193
:107AB000440D511D47FC5A95588F4F8B69817A812F
:107AC000660D711D67FC7A957E876D877989C7166B
:107AD00008F051CF2C2D30E04D815E81420F531FB5
:107AE000A985BA854A9FC0014B9F900D5A9F900D62
:107AF0001124FC01E80DF91DF88BEF87852D612C11
:107B00004F89588D420F531F5E8B4D8B671408F0C1
:107B100050C044244394480E877041F4C10101963B
:107B2000EB89FC89E20DF31DD4901C01D7FE19C02E
:107B3000A98DBA8DED91FC91662D70E0B1E0BB127C
:107B400019C0AB1217C02D853E85620F731F0484C8
:107B5000F585E02D2F8138854D895E89898D9A8D37
:107B60000995DD0C6394842DD1CF1E821D821C8269
:107B70001B8288CF4B815C81640F751FAB85BC85F0
:107B80006A9FC0016B9F900D7A9F900D11246981AF
:107B90007A81680F791F0684F785E02DEF80F884DD
:107BA00009851A859D014F855889898D9A8D09957A
:107BB000D8CF570CC3948ACF6A960FB6F894DEBF1D
:107BC0000FBECDBFDF91CF911F910F91FF90EF902E
:107BD000DF90CF90BF90AF909F908F907F906F90ED
:107BE0005F904F903F902F9008958F929F92AF9209
:107BF000CF92EF92FF920F931F93CF93DF93EC01FD
:107C0000262F898D9A8D009709F051C06A30D1F4E2
:107C10001D861C868D8948E0849F900111248E85E5
:107C20009F85820F931F9F878E8781E090E0DF9171
:107C3000CF911F910F91FF90EF90CF90AF909F90B9
:107C40008F9008956D3089F3CC88AD888F89882313
:107C5000C1F08C859D8536E0C39E800D911D112459
:107C6000488559854817590764F44E855F851D86F8
:107C70001C8638E0A39EC0011124840F951F9F87A6
:107C80008E87EA88FB88088919894E855F856C850F
:107C90007D85CE010E94D03B2C898C859D8546E058
:107CA000249F800D911D11249D878C87BECF6A3043
:107CB00069F41D861C86FC013896E4912D898E8519
:107CC0009F85E29F800D911D1124ADCF6D3009F489
:107CD000ACCFFC0134963491631708F4A6CF3296EA
:107CE000E491E61708F4A1CFFC01329685909490B8
:107CF000462F431B342F47E0349F800C911C1124E6
:107D0000F401329634913196E4913323A9F1EE23B4
:107D100099F1CC88F4013596E491AD884F894423DC
:107D200001F10E2E000CFF0BE30FF11DCE9EA00102
:107D3000CF9E500D11246C857D85460F571F688599
:107D40007985641775076CF44E855F851D861C86E2
:107D5000FC013896E491AE9E400D511D11245F87C1
:107D60004E87EA88FB88088919894E855F856C856E
:107D70007D85CE010E94D03BF4013496E4912C899C
:107D80008C859D85E29F800D911D11248DCF611101
:107D900001C061E0FC01648B411101C041E0FC01C4
:107DA000458B0895462F0C94C73E8091C7068823C3
:107DB00061F09FB7F8942091C7068091C5062130E5
:107DC00019F489BF9FBF08958FBF0895FC0177FD07
:107DD00064C080859185681779070CF05EC057FDF7
:107DE0005CC082859385481759070CF056C0868978
:107DF0008230B1F0833029F1813041F48481958162
:107E0000841B950BAB01BC01615071092130310518
:107E100009F108F443C02230310509F463C0089524
:107E200084819581DC01A61BB70BBD0161507109EE
:107E300086819781DC01A41BB50BAD01415051092E
:107E4000E5CF86819781861B970BBA01AC01415023
:107E50005109DCCFCA0157FD0796A3E09595879598
:107E6000AA95E1F7A481B5818A9F90018B9F300D7F
:107E70009A9F300D1124620F731F078CF0A1E02D23
:107E8000E60FF71F4770552721E030E001C0220FB1
:107E90004A95EAF78081822B80830895CA0157FDB5
:107EA000079633E0959587953A95E1F7A481B581DA
:107EB0008A9F90018B9F300D9A9F300D1124620F85
:107EC000731F078CF0A1E02DE60FF71F47705527B1
:107ED00081E090E001C0880F4A95EAF78095908193
:107EE0008923DACFCA0157FD079623E09595879538
:107EF0002A95E1F7A481B5818A9F90018B9F300D6F
:107F00009A9F300D1124620F731F078CF0A1E02D92
:107F1000E60FF71F4770552721E030E001C0220F20
:107F20004A95EAF780818227B7CF4F925F926F928E
:107F30007F928F929F92AF92BF92CF92DF92EF92F9
:107F4000FF920F93CF93DF93CDB7DEB73C012901AA
:107F500050E070E00E942F3985E792E0F3019183B1
:107F60008083148E138E4114510421F489EC482E21
:107F700086E0582EF301568E458E10A2178E8FEF95
:107F800084A385A386A387A300A7C5AAD6AAE7AA28
:107F9000F0AE81AE92AEA3AEB4AE80E586AF17AEC2
:107FA000DF91CF910F91FF90EF90DF90CF90BF9036
:107FB000AF909F908F907F906F905F904F900895BB
:107FC00025E732E0FC0131832083878D90A1009763
:107FD00011F00C946F5008951F93CF93DF93EC0131
:107FE0008D8D9E8D009711F1162F69A1062E000C24
:107FF000770B0E9479348D8D9E8DDC01ED91FC9183
:108000000190F081E02D60E009958D8D9E8DDC0161
:10801000ED91FC910190F081E02D612F09958D8DFE
:108020009E8DDF91CF911F910C948E34ADA5BEA58E
:108030009C918BA9809589238C938B8D9C8D892B0A
:1080400031F0862FDF91CF911F910C94530928E0D6
:1080500030E080E8A9A5BAA599A9462F4823C1F028
:108060004C91942B9C93ABA5BCA59C914AA9942BB5
:108070009C93ABA5BCA54C919AA9909594239C93F5
:1080800086952150310931F7DF91CF911F910895E5
:108090004C9190959423E6CF1F93CF93DF93EC01FF
:1080A000162F8D8D9E8D0097C9F04DA95EA96FA9E1
:1080B00078AD0E946B3466EA111167EACE010E9426
:1080C000EC3F8D8D9E8D0097C9F049AD5AAD6BADDB
:1080D0007CADDF91CF911F910C946B348B8D9C8D77
:1080E000892B21F08EAD9FAD0E94C321EFA5F8A989
:1080F00090818CA9809589238083DDCFEFA5F8A995
:1081000080819CA9892B80838B8D9C8D892B29F064
:10811000DF91CF911F910C94D53EDF91CF911F91AC
:108120000895CF92DF92EF92FF921F93CF93DF9348
:10813000EC016B01142F8D8D9E8D009709F44FC0BB
:1081400069A1062E000C770B0E9479348D8D9E8DCF
:10815000DC01ED91FC910190F081E02D60E009954A
:108160007601CC24C394D12C11508D8D9E8D1F3F50
:1081700069F1B0E2CB16D104B8F00E948E3469A147
:10818000062E000C770B8D8D9E8D0E9479348D8D7F
:108190009E8DDC01ED91FC910190F081E02D60E07D
:1081A0000995CC24C394D12C8D8D9E8DF7016491BB
:1081B000DC01ED91FC910190F081E02D0995BFEF7C
:1081C000CB1ADB0AEFEFEE1AFE0ACECFDF91CF918A
:1081D0001F91FF90EF90DF90CF900C948E34EDA51F
:1081E000FEA590818BA98095892380837B01115006
:1081F00070F1F70184912B8D3C8D232B31F00E947F
:108200005309FFEFEF1AFF0AF2CF28E030E040E811
:10821000E9A5FAA599A9582F5423A9F05081952BC7
:108220009083EBA5FCA590815AA9952B9083EBA593
:10823000FCA550819AA9909595239083469521504D
:10824000310931F7DECF508190959523E9CFDF9149
:10825000CF911F91FF90EF90DF90CF900895FC0198
:10826000868197819C01295F3F4F37FF02C0295FBC
:108270003F4F83E0359527958A95E1F78481958175
:10828000289FA001299F500D389F500D112470E0A8
:1082900060E0878D90A10C9404528F929F92AF92D0
:1082A000BF92CF92DF92EF92FF920F931F93CF93E3
:1082B000DF93EC01862EB42EA22E902E8F8D98A1E6
:1082C000892B39F1CE010E942F418E819F816C81D3
:1082D0007D81813291050CF046C0AC0140525109BC
:1082E00057FF02C04F5F5F4F559547956357710920
:1082F00077FF02C06F5F7F4F75956795CC24C3945D
:10830000D12CA0E2EA2EF12C03E710E023EC3AE0B6
:1083100045C02E813F81C901079697FD079623E04E
:10832000959587952A95E1F72C813D81AC01429F77
:10833000C001439F900D529F900D11240E94D34F76
:1083400098A38F8F892B09F0BDCF80E0DF91CF916B
:108350001F910F91FF90EF90DF90CF90BF90AF9063
:108360009F908F900895AC014054510957FF02C06F
:108370004F5F5F4F559547956255710977FF02C072
:108380006F5F7F4F75956795CC24C394D12C80E4A3
:10839000E82EF12C02E510E023EA3CE0CE010E9439
:1083A000383B8AA22D8D3E8D2115310509F4A2C0DE
:1083B0009B2DB11006C08E819F81809709F098C0D7
:1083C0009CE399A3992009F43FC1C9010E94593443
:1083D000AA20F1F088A587FD1BC061E00E94D74864
:1083E00061E088A50E94134961E070E080E090E0C0
:1083F0000E94C74760E088A50E9413496AE070E0C8
:1084000080E090E00E94C74761E088A50E94134980
:108410002D8D3E8D2115310509F4E6C04DA95EA9CB
:108420006FA978ADC9010E946B3444E06FEB7AE02C
:10843000CE010E9491406E816150CE010E94EC3FBE
:1084400044E06BEB7AE0CE010E9491408AA160E1AA
:10845000813009F064E1CE010E94EC3F44E067EB1B
:108460007AE0CE010E9491408FE88DAF8C819D8192
:108470008038910509F0CAC08E819F8180349105B2
:1084800009F0D0C08AA1813009F0BEC08FE98DAF5C
:1084900012E16AEDCE010E94EC3F612FCE010E94F5
:1084A000EC3F61E8CE010E94EC3F6DADCE010E9431
:1084B000EC3F69EDCE010E94EC3F8AA162E281307F
:1084C00009F061EFCE010E94EC3F46E061EB7AE0FB
:1084D000CE010E9491408D8D9E8D009709F4A6C01B
:1084E00049AD5AAD6BAD7CAD0E946B3481E02ECFAF
:1084F0009DE367CF61E08EA10E94D74861E08FA124
:108500000E94D7488EA1082E000C990BFC01E35362
:10851000F04FE491F0E0EE0FFF1FEE5EFF4E25916D
:1085200034913EA72DA7FC01E856F04FE491EBAB48
:108530008FA1082E000C990BFC01E353F04FE4913E
:10854000F0E0EE0FFF1FEE5EFF4EA591B491B8ABC9
:10855000AFA7FC01E856F04FE491ECAB8C91E82B0F
:10856000EC938B8D9C8D892B31F0992009F430CFC1
:108570000E946B332DCF61E08CA10E94D74861E04F
:108580008DA10E94D7488CA1082E000C990BFC01EC
:10859000E353F04FE491F0E0EE0FFF1FEE5EFF4E6D
:1085A000259134913AA729A7FC01E856F04FE491B0
:1085B000E9AB8DA1082E000C990BFC01E353F04FA1
:1085C000E491F0E0EE0FFF1FEE5EFF4EA591B49137
:1085D000BCA7ABA7FC01E856F04FE491EAAB8C9145
:1085E000E095E823EC93F4CE8B8D9C8D892B21F0C4
:1085F0008EAD9FAD0E94C321EFA5F8A990818CA9F3
:1086000080958923808311CF8FEC41CF80369105EF
:1086100049F48E819F81409729F48AA1813021F409
:1086200080E18DAF12E035CF8FEAFBCFEFA5F8A93F
:1086300080819CA9892B80838B8D9C8D892B09F44B
:1086400055CF0E94D53E52CFA110C4CEE7CE0F9396
:108650001F93CF93DF93DC0157FD46C016968D9193
:108660009C911797481759070CF03EC077FF04C03C
:10867000260F371F70E060E01496CD91DC911597BE
:10868000CB01820F931FC817D9071CF49E01261B2C
:10869000370B1216130644F5FA0157FD379683E09F
:1086A000F595E7958A95E1F7EC9FC001ED9F900D58
:1086B000FC9F900D1124680F791F5F96ED91FC913E
:1086C000E60FF71F4770552781E090E001C0880F43
:1086D0004A95EAF7482F0130110559F0A8F02E0FFE
:1086E0003F1F02301105E1F0DF91CF911F910F91F3
:1086F00008952E0F3F1FE217F307B1F38191DF01B9
:108700001197842B8C93F7CF80952E0F3F1FE21784
:10871000F30751F39191DF01119798239C93F7CFC1
:10872000E217F30709F38191DF01119784278C93F6
:10873000F7CFEF92FF920F931F93CF93DF93EC014C
:1087400077FD76C0EC80FD806E157F050CF070C063
:1087500057FF04C0240F351F50E040E08E819F81F9
:10876000FA01E20FF31F8E179F071CF49C01241BD4
:10877000350B121613060CF05BC0922F842F8695D2
:10878000869586958E9DD0018F9DB00D11246A0F20
:108790007B1FAF8DB8A1A60FB71F477049F188E0C6
:1087A000841B482F682F70E0FB01E755F54FE491DB
:1087B000281708F063C0621B71092FEF30E002C078
:1087C000359527956A95E2F7E2230130110539F0D6
:1087D000B0F10230110561F58C91E82702C08C914F
:1087E000E82BEC93941720F12C813D81A20FB31F4D
:1087F000E92FE41BE83078F00230110521F58E2FC7
:108800009C9190959C932C813D81A20FB31F885021
:108810008830B0F7E770EE2359F0F0E0EF55F54FF0
:10882000E49101301105F9F010F10230110519F150
:10883000DF91CF911F910F91FF90EF900895E095F8
:108840008C91E823CECF81E00115110509F480E079
:1088500081959E2F8C932C813D81A20FB31F985040
:108860009830C0F7D7CF8C91E82BEC93E1CFE0950F
:108870008C91E823FACF8C91E827F7CF01301105CE
:1088800009F4ADCFE0F20230110509F4A5CFAE0D29
:10889000BF1DAECF0F931F93FA01DC0156964C918A
:1088A0005697423089F0433039F14130F9F414964B
:1088B0004D915C91DA01AE1BBF0BFD013197AB010D
:1088C000BF010E94994315C016964D915C91DA0143
:1088D000AE1BBF0BFD013197DC0114964D915C91ED
:1088E000DA01A61BB70BBD01621B730BAF010E941F
:1088F00027431F910F91089516964D915C91DA01CF
:10890000A61BB70BBD01621B730BD9CF0F931F932F
:10891000FA01DC0156964C915697423091F0433063
:1089200049F1413009F514964D915C91DA01AE1B85
:10893000BF0BFD01E21BF30BAB01BF010E942743FC
:1089400016C014964D915C91DA01A61BB70BBD01C0
:1089500061507109DC0116964D915C91DA01AE1BF4
:10896000BF0BFD01E21BF30BAF010E9499431F9166
:108970000F91089516964D915C91DA01A61BB70BE5
:10898000BD0161507109D8CFCF92DF92EF92FF9273
:108990000F931F93CF93DF93EC018D8D9E8D0097E6
:1089A00009F46EC04DA95EA96FA978AD0E946B3421
:1089B00045E06CE97AE0CE010E9491406C81615003
:1089C000CE010E94EC3F2E813F81C901079697FDA1
:1089D000079623E0959587952A95E1F72C813D81AF
:1089E000829F7001839FF00C929FF00C11240F8DD9
:1089F00018A18D8D9E8DE00EF11E009709F465C0C3
:108A000069A1062E000C770B0E9479348D8D9E8D06
:108A1000DC01ED91FC910190F081E02D60E409957D
:108A2000680101E010E08D8D9E8DEC14FD04C1F114
:108A300000321105B0F00E948E3469A1062E000CA0
:108A4000770B8D8D9E8D0E9479348D8D9E8DDC01EE
:108A5000ED91FC910190F081E02D60E4099501E039
:108A600010E08D8D9E8DF60161916F01DC01ED911D
:108A7000FC910190F081E02D09950F5F1F4FD3CF3E
:108A80008B8D9C8D892B21F08EAD9FAD0E94C321D3
:108A9000EFA5F8A990818CA980958923808388CF40
:108AA0000E948E348D8D9E8D009709F443C049AD90
:108AB0005AAD6BAD7CADDF91CF911F910F91FF90BF
:108AC000EF90DF90CF900C946B34EDA5FEA58081E4
:108AD0009BA9892B8083E016F10621F3F80181918F
:108AE0008F012B8D3C8D232B19F00E945309F3CF5E
:108AF00028E030E040E8E9A5FAA599A9582F5423C9
:108B0000A9F05081952B9083EBA5FCA590815AA9E3
:108B1000952B9083EBA5FCA550819AA99095952360
:108B2000908346952150310931F7D5CF50819095EA
:108B30009523E9CFEFA5F8A980819CA9892B808393
:108B40008B8D9C8D892B51F0DF91CF911F910F91CF
:108B5000FF90EF90DF90CF900C94D53EDF91CF91B6
:108B60001F910F91FF90EF90DF90CF900895CF93DA
:108B7000DF93EC0160E08E810E94134981E090E078
:108B80000E94004861E08E810E94134981E090E0DC
:108B90000E94004860E08E810E94134984E690E0C4
:108BA000DF91CF910C940048CF92DF92EF92FF9229
:108BB0000F931F93CF93DF936C017C0187E0E80E46
:108BC000F11CD0E0C0E0062F10E0B8010C2E02C06E
:108BD000759567950A94E2F76170F70181917F01BD
:108BE0000E9413492196C430D10579F7C601DF915F
:108BF000CF911F910F91FF90EF90DF90CF900C9449
:108C0000B745CF92DF92EF92FF920F931F93CF93CE
:108C1000DF936C017C0187E0E80EF11CD0E0C0E03E
:108C2000062F10E0B8010C2E02C0759567950A94C6
:108C3000E2F76170F70181917F010E94134921964B
:108C4000C830D10579F7C601DF91CF911F910F91FF
:108C5000FF90EF90DF90CF900C94B7451F93CF9388
:108C6000DF93EC01162F642F8C810E9413498D81B4
:108C70008F3F19F060E00E9413498F85612F84FFB8
:108C800006C0CE01DF91CF911F910C94014670E098
:108C900084E0759567958A95E1F7CE010E94D445E9
:108CA000612FCE01DF91CF911F910C94D44540E00C
:108CB0000C942E4661E00E94574680ED97E00C949C
:108CC0000048443008F043E0FC012389421710F0CB
:108CD0004FEF420FFC01E40FF11D2489620F606821
:108CE0000C945746FC016089262F2460208B6C6011
:108CF0000C9457460F931F93CF93DF93EC014230B0
:108D000018F08F8588608F874B8B1C8A80E48D8B51
:108D10006E8B605C6F8B222329F0413019F48F85B4
:108D200084608F8761E08C810E94D7488D818F3F5E
:108D300019F061E00E94D74861E08E810E94D74817
:108D40008E0198012C1B3D0B8F8584FD0DC084E0A6
:108D500090E00F5F1F4F281739074CF461E0F801CE
:108D600086810E94D748EDCF88E090E0F2CF80E581
:108D700093EC0E94004860E08C810E94134960E0FF
:108D80008E810E9413498D818F3F19F060E00E940F
:108D900013496F8564FD33C063E0CE010E94D44562
:108DA00084E991E10E94004863E0CE010E94D4452D
:108DB00084E991E10E94004863E0CE010E94D4451D
:108DC00086E990E00E94004862E0CE010E94D4450E
:108DD0006F856062CE010E94574684E0888BCE0189
:108DE0000E947246CE010E945A4682E0898B66E05C
:108DF000CE01DF91CF911F910F910C945746606285
:108E0000CE010E94574684E991E10E9400486F8597
:108E10006062CE010E94574686E990E00E940048B9
:108E20006F856062CE010E945746D2CFCF92EF92FB
:108E30000F93FC011382128281EA92E09183808376
:108E400064838FEF8583468327830087E186C2860C
:108E50001386148615861686178620E041E060E1A9
:108E6000CF010F91EF90CF900C947A46FC0160896E
:108E70006E7F608B68600C945746FC016089262FDA
:108E80002160208B69600C94574641E00E942E4679
:108E900081E090E008951F920F920FB60F92112477
:108EA0002F933F938F939F93AF93BF9380917407BA
:108EB00090917507A0917607B0917707309173076D
:108EC00023E0230F2D3768F126E8230F0296A11D1A
:108ED000B11D209373078093740790937507A09337
:108EE0007607B093770780916F0790917007A091F4
:108EF0007107B09172070196A11DB11D80936F0794
:108F000090937007A0937107B0937207BF91AF91D0
:108F10009F918F913F912F910F900FBE0F901F90B7
:108F200018950196A11DB11DD4CF2FB7F89460916B
:108F300074077091750780917607909177072FBF1E
:108F400008953FB7F89480916F0790917007A091B2
:108F50007107B091720722B706B600FE05C02F3F19
:108F600019F00196A11DB11D3FBFBA2FA92F982F4F
:108F70008827BC01CD01620F711D811D911D42E04A
:108F8000660F771F881F991F4A95D1F708958F9212
:108F90009F92AF92BF92CF92DF92EF92FF926B01BE
:108FA0007C010E94A1474B015C01C114D104E10482
:108FB000F104E9F00E948D4F0E94A14768197909D8
:108FC0008A099B09683E73408105910570F321E091
:108FD000C21AD108E108F10888EE880E83E0981ED5
:108FE000A11CB11CC114D104E104F10429F7FF90C4
:108FF000EF90DF90CF90BF90AF909F908F900895AB
:109000008230910538F0880F991F880F991F0597B6
:109010000197F1F70895789483B78C6483BF87B77D
:10902000816087BF82E08EBD8EB581608EBD8FB5B9
:1090300081608FBD85B5846085BD85B5806485BD43
:10904000EAE8F0E0808183608083EBE8F0E08081F3
:109050008160808387E886B91AB808951F93CF93FB
:10906000DF93182FEB0161E00E94D748209739F475
:1090700060E0812FDF91CF911F910C941349CF3F76
:10908000D10511F461E0F5CFE12FF0E0ED59F04F9B
:10909000E491E150EC3008F050C0F0E0EE5AF74BAC
:1090A0000C94B04F5E485E489D4866486C487248D4
:1090B0007A489D489D487F488948934883B7806295
:1090C00083BFC1BFDF91CF911F9108958FB5806895
:1090D0008FBDDBBDCABDF6CF8FB580628FBDD9BD58
:1090E000C8BDF0CF8FB588608FBDD0937900C09395
:1090F0007800E8CF85B5806285BDC3BDE3CF8091A0
:109100008B00806880938B00D0938700C09386008B
:10911000D9CF80918B00806280938B00D0938500A3
:10912000C0938400CFCF80918B00886080938B00A8
:10913000D0938300C0938200C5CFC038D1050CF016
:10914000A1CF96CF81508C3088F5E82FF0E0E5551F
:10915000F74B0C94B04FD348D348D648B748BB48D8
:10916000BE48C148D648D648C548CB48CF488FB539
:109170008F778FBD08958FB58F7DFBCF8FB5877F9C
:10918000F8CF85B58F7D85BD089580918B008F7751
:1091900080938B00089580918B008F7DF9CF809113
:1091A0008B00877FF5CF83B78F7D83BF0895CF93E3
:1091B000DF9390E0FC01E856F04F24918353904FE9
:1091C000FC0184918823C9F090E0880F991FFC016D
:1091D000EE5DFF4EA591B491FC01EE5EFF4EC59190
:1091E000D49161110DC09FB7F8948C912095822382
:1091F0008C938881282328839FBFDF91CF91089586
:10920000623051F49FB7F8943C91822F809583236C
:109210008C93E8812E2BEFCF8FB7F894EC912E2B07
:109220002C938FBFEACF1F93CF93DF93282F30E08B
:10923000F901ED59F04F8491F901E856F04FD491BE
:10924000F901E353F04FC491CC23A9F0162F8111FB
:109250000E94A248EC2FF0E0EE0FFF1FEE5EFF4EE3
:10926000A591B4918FB7F894EC91111108C0D095E5
:10927000DE23DC938FBFDF91CF911F910895DE2B0A
:10928000F8CFCF93DF93282F30E0F901ED59F04F5D
:109290008491F901E856F04FD491F901E353F04F6E
:1092A000C491CC23A1F081110E94A248EC2FF0E0E0
:1092B000EE0FFF1FEE5FFF4EA591B491EC91ED23F1
:1092C00081E090E009F480E0DF91CF91089580E0A3
:1092D00090E0FACFFC01918D228D892F90E0805C87
:1092E0009F4F821B91098F7399270895FC01918DDF
:1092F000828D981731F0828DE80FF11D858D90E0F9
:1093000008958FEF9FEF0895FC01918D828D98173E
:1093100061F0A28DAE0FBF2FB11D5D968C91928D25
:109320009F5F9F73928F90E008958FEF9FEF089556
:10933000FC01538D448D252F30E0842F90E0821B5B
:10934000930B541710F0CF9608950197089589E074
:109350009BE4892B49F080E090E0892B29F00E9462
:10936000094B81110E94000080E090E0892B49F0B8
:1093700080E090E0892B29F00E94000081110C947C
:1093800000000895FC01A48DA80FB92FB11DA35AA8
:10939000BF4F2C91848D90E001968F739927848F15
:1093A000A689B7892C93A089B1898C918370806438
:1093B0008C93938D848D981306C00288F389E02DD9
:1093C00080818F7D80830895CF93DF93EC01888D1A
:1093D0008823B9F0AA89BB89E889F9898C9185FD30
:1093E00003C0808186FD0DC00FB607FCF7CF8C91BE
:1093F00085FFF2CF808185FFEDCFCE010E94C2496B
:10940000E9CFDF91CF910895EF92FF920F931F93D1
:10941000CF93DF93EC0181E0888F9B8D8C8D981327
:109420001AC0E889F989808185FF15C09FB7F89433
:10943000EE89FF896083E889F9898081837080647F
:1094400080839FBF81E090E0DF91CF911F910F91CA
:10945000FF90EF900895F62E0B8D10E00F5F1F4FD9
:109460000F731127E02E8C8D8E110CC00FB607FCE8
:10947000FACFE889F989808185FFF5CFCE010E9476
:10948000C249F1CFEB8DEC0FFD2FF11DE35AFF4FD9
:10949000F0829FB7F8940B8FEA89FB898081806204
:1094A000CFCFCF92DF92EF92FF921F93CF93DF93B4
:1094B000EC016A017B01122FE889F98982E080833F
:1094C000C11481EED806E104F104A1F060E079E076
:1094D0008DE390E0A70196010E948E4F2150310943
:1094E000410951095695479537952795211580E1F2
:1094F000380798F0E889F989108260E874E88EE10D
:1095000090E0A70196010E948E4F21503109410938
:1095100051095695479537952795EC85FD853083FC
:10952000EE85FF852083188EEC89FD891083EA89FA
:10953000FB89808188698083EA89FB8980818F7DAE
:109540008083DF91CF911F91FF90EF90DF90CF90BC
:1095500008951F920F920FB60F9211240BB60F921F
:109560002F938F939F93EF93FF93E0918807F09150
:1095700089078081E0918E07F0918F0782FD1DC0E1
:109580009081809191078F5F8F732091920782174E
:1095900041F0E0919107F0E0E858F84F958F809303
:1095A0009107FF91EF919F918F912F910F900BBE9B
:1095B0000F900FBE0F901F9018958081F2CF1F92D1
:1095C0000F920FB60F9211240BB60F922F933F9369
:1095D0004F935F936F937F938F939F93AF93BF93BB
:1095E000EF93FF9388E797E00E94C249FF91EF91C4
:1095F000BF91AF919F918F917F916F915F914F91AB
:109600003F912F910F900BBE0F900FBE0F901F90A8
:10961000189588E797E00E946A4921E0892B09F4B0
:1096200020E0822F0895E8E7F7E01382128288EEA7
:1096300093E0A0E0B0E084839583A683B7838DEAAE
:1096400092E09183808380E990E09587848789E226
:1096500090E0978786878BE290E0918B808B8AE2FF
:1096600090E0938B828B85E990E0958B848B8CE2E4
:1096700090E0978B868B118E128E138E148E089528
:10968000AF92BF92CF92DF92EF92FF920F931F9310
:10969000CF93DF936C017B018B01040F151FEB014E
:1096A0005E01AE18BF08C017D10759F06991D60105
:1096B000ED91FC910190F081E02DC6010995892B77
:1096C00079F7C501DF91CF911F910F91FF90EF9036
:1096D000DF90CF90BF90AF900895FB0101900020E4
:1096E000E9F73197AF01461B570BDC01ED91FC9177
:1096F0000280F381E02D0994EF92FF920F931F9364
:10970000CF93DF938C017B01D0E0C0E0F701EC0F39
:10971000FD1F6491662361F0D801ED91FC910190E9
:10972000F081E02DC8010995892B11F02196EECF2B
:10973000CE01DF91CF911F910F91FF90EF9008958F
:10974000DB0114964D915C9115976D917C91DC0134
:10975000ED91FC910280F381E02D09946115710572
:1097600011F00C946D4B90E080E00895DC01ED91D8
:10977000FC910190F081E02D09946BEB72E00C9468
:109780006D4B0F931F93CF93DF93EC010E947C4BA3
:109790008C01CE010E94BD4B800F911FDF91CF91B4
:1097A0001F910F9108950F931F93CF93DF93EC01B7
:1097B0000E94A04B8C01CE010E94BD4B800F911FD7
:1097C000DF91CF911F910F9108950F931F93CF9326
:1097D000DF938C01D0E0C0E06115710519F00E94A3
:1097E0006D4BEC01C8010E94BD4B8C0F9D1FDF919A
:1097F000CF911F910F9108958F929F92AF92BF9238
:10980000EF92FF920F931F93CF93DF93CDB7DEB705
:10981000A1970FB6F894DEBF0FBECDBF7C01FA0151
:10982000CB0119A2223008F42AE08E010F5D1F4FF0
:10983000822E912CB12CA12CBF01A50194010E9474
:109840008E4FF901CA016A300CF5605DD8016E9344
:109850008D01232B242B252B79F790E080E01097A6
:1098600021F0BD01C7010E946D4BA1960FB6F8947F
:10987000DEBF0FBECDBFDF91CF911F910F91FF9043
:10988000EF90BF90AF909F908F900895695CDECF6E
:109890002115310541F4DC01ED91FC910190F0813D
:1098A000E02D642F09940C94FC4B9A01462F50E054
:1098B00070E060E00C94484C0F931F93CF93DF93BC
:1098C000EC010E94554C8C01CE010E94BD4B800FD3
:1098D000911FDF91CF911F910F9108959A01AB01D4
:1098E00070E060E00C94484C0F931F93CF93DF938C
:1098F000EC010E946E4C8C01CE010E94BD4B800F8A
:10990000911FDF91CF911F910F910895982F862F6E
:1099100008950895FC0180819181009711F00C94C5
:109920006F500895CF93DF93EC0188819981009760
:1099300011F00E946F50198218821D821C821B82B6
:109940001A82DF91CF9108950F931F93CF93DF93E6
:10995000EC018B016F5F7F4F888199810E94F850E5
:10996000009751F0998388831B830A8381E0DF91FC
:10997000CF911F910F91089580E0F9CFCF93DF939E
:10998000EC0188819981892B49F08A819B81861716
:10999000970720F081E0DF91CF910895CE010E94DA
:1099A000A44C8823C1F38C819D81892B99F7E88190
:1099B000F9811082EFCFEF92FF920F931F93CF9315
:1099C000DF93EC017B018A01BA010E94BE4C811138
:1099D0000BC0CE010E94924CCE01DF91CF911F911E
:1099E0000F91FF90EF9008951D830C83B70188813C
:1099F00099810E941F52F0CFFC01118210821382C4
:109A00001282158214826115710551F0FB010190DB
:109A10000020E9F73197AF01461B570B0C94DB4C44
:109A20000895FB0101900020E9F73197AF01461B33
:109A3000570B0C94DB4C0F931F93CF93DF93CDB751
:109A4000DEB729970FB6F894DEBF0FBECDBF8C01ED
:109A5000862FF801118210821382128215821482DD
:109A600050E0BE016F5F7F4F90E00E944F52BE01F9
:109A70006F5F7F4FC8010E94114D29960FB6F89471
:109A8000DEBF0FBECDBFDF91CF911F910F91089523
:109A90000F931F93CF93DF93CDB7DEB761970FB6C8
:109AA000F894DEBF0FBECDBF8C01CB01F80111824F
:109AB0001082138212821582148250E0BE016F5F01
:109AC0007F4F0E944F52BE016F5F7F4FC8010E94BF
:109AD000114D61960FB6F894DEBF0FBECDBFDF917A
:109AE000CF911F910F910895EF92FF920F931F93C3
:109AF000CF93DF93EC017B018A01BA010E94BE4C37
:109B000081110BC0CE010E94924CCE01DF91CF910A
:109B10001F910F91FF90EF9008951D830C83B70163
:109B2000888199810E94DE51F0CF0F931F93CF93CC
:109B3000DF938C01EB01FC0180819181009701F1A1
:109B40006881798161157105C9F029E83CE4232B0E
:109B5000A9F0428153812C813D814217530770F057
:109B60000E941F528C819D81F801958384831D8200
:109B70001C82DF91CF911F910F9108950E946F5029
:109B800088819981F801918380838A819B81938365
:109B900082838C819D8195838483198218821B82A4
:109BA0001A82E5CFFC011182108213821282158283
:109BB00014820C94954DCF93DF93EC01FB01861733
:109BC000970749F0608171816115710541F0448109
:109BD00055810E94DB4CCE01DF91CF9108950E9408
:109BE000924CF9CFFC0111821082138212821582ED
:109BF00014820C94DB4DCF93DF93EC01611571055A
:109C000031F00E94114DCE01DF91CF9108950E9455
:109C1000924CF9CF0F931F93CF93DF93EC018B01FD
:109C20006115710571F0CB010E94E551AC01B801DD
:109C3000CE010E94744DCE01DF91CF911F910F9103
:109C400008950E94924CF7CFFC011182108213827A
:109C50001282158214820C940A4EEF92FF920F9397
:109C60001F93CF93DF936115710541F480E0DF917D
:109C7000CF911F910F91FF90EF90089541155105DD
:109C8000B1F07B01EC010C811D81040F151FB8019F
:109C90000E94BE4C882351F3288139818C819D819B
:109CA000B701820F931F0E941F521D830C8381E016
:109CB000DECFFB0144815581608171810C942D4E72
:109CC0006115710551F0FB0101900020E9F7319712
:109CD000AF01461B570B0C942D4E80E00895CF9397
:109CE000DF9300D0CDB7DEB769831A8241E050E040
:109CF000BE016F5F7F4F0E942D4E0F900F90DF913E
:109D0000CF910895CF93DF93EC01FB0144815581FE
:109D1000608171810E942D4E811103C0CE010E948D
:109D2000924CCE01DF91CF910895CF93DF93EC0158
:109D30006115710539F4CE010E94924CCE01DF917C
:109D4000CF910895FB0101900020E9F73197AF0111
:109D5000461B570B0E942D4E882369F3EFCFFC0161
:109D600024813581232B31F421E0FB01672B49F459
:109D7000822F0895808191816115710539F421E068
:109D8000FC0180818823A1F320E0F2CF0E941652CB
:109D900021E0892B69F3F8CFFC0124813581FB0197
:109DA0004481558124173507A0F0FC018081918101
:109DB000009779F0FB01608171816115710549F0AF
:109DC000241B350B820F931F0E94165221E0892B12
:109DD00009F020E0822F0895AF92BF92CF92DF92D8
:109DE000EF92FF920F931F93CF93DF936B01EA01E2
:109DF000FB01448155814115510561F1FC0124812C
:109E000035812115310531F12417350718F1C217B5
:109E1000D30710F0E9012197FC0100811181C801ED
:109E2000AA24AA94BB24BA947801EC0EFD1EE8166D
:109E3000F906A0F0F601608171810E943552009709
:109E400069F09C01201B310BC217D30708F05901A0
:109E50000196EDCFAA24AA94BB24BA94C501DF9140
:109E6000CF911F910F91FF90EF90DF90CF90BF9017
:109E7000AF900895FC0144815581FB012481358117
:109E8000421B530B0C94EC4ECF93DF93DC011496E2
:109E9000ED91FC916E177F0728F54115510511F1E1
:109EA0009F01261B370B4217530708F49A01DB0169
:109EB000EC0188819981E21BF30BFD83EC83AF01F8
:109EC000461B570B260F371FBC01620F731F8A0FEB
:109ED0009B1F0E942652E881F9818C819D81E80FA9
:109EE000F91F1082DF91CF9108954FEF5FEF0C942F
:109EF000444F0E94D9510E94794F08950E940B4807
:109F00000E947D4F0E947B1BC7EAD9E40E94F31C8C
:109F10002097E1F30E94A749F9CF0895A1E21A2EF4
:109F2000AA1BBB1BFD010DC0AA1FBB1FEE1FFF1FFD
:109F3000A217B307E407F50720F0A21BB30BE40B4D
:109F4000F50B661F771F881F991F1A9469F7609594
:109F50007095809590959B01AC01BD01CF0108954E
:109F6000EE0FFF1F0024001C0BBE0790F691E02DA2
:109F70000994A29FB001B39FC001A39F700D811DE2
:109F80001124911DB29F700D811D1124911D089502
:109F90000E94B94FA59F900DB49F900DA49F800D76
:109FA000911D112408950F931F93CF93DF93823057
:109FB000910510F482E090E0E0911708F091180804
:109FC00030E020E0B0E0A0E0309799F421153105B1
:109FD00009F44AC0281B390B24303105D8F58A8191
:109FE0009B816115710589F1FB0193838283FE01D9
:109FF00011C0408151810281138148175907E0F057
:10A000004817590799F4109761F012960C9312971C
:10A0100013961C933296CF01DF91CF911F910F9130
:10A0200008950093170810931808F4CF21153105EF
:10A0300051F04217530738F0A901DB019A01BD0125
:10A04000DF01F801C1CFEF01F9CF90931808809399
:10A050001708CDCFFE01E20FF31F81939193225099
:10A06000310939832883D7CF2091150830911608FC
:10A07000232B41F420910201309103013093160803
:10A08000209315082091000130910101211531051F
:10A0900041F42DB73EB74091040150910501241BB6
:10A0A000350BE0911508F0911608E217F307A0F4BC
:10A0B0002E1B3F0B2817390778F0AC014E5F5F4F1E
:10A0C0002417350748F04E0F5F1F50931608409332
:10A0D0001508819391939FCFF0E0E0E09CCFCF9360
:10A0E000DF930097E9F0FC01329713821282A0916E
:10A0F0001708B0911808ED0130E020E01097A1F4A6
:10A1000020813181820F931F20911508309116080C
:10A110002817390709F061C0F0931608E093150875
:10A12000DF91CF910895EA01CE17DF07E8F54A8164
:10A130005B819E0141155105B1F7E901FB83EA837B
:10A1400049915991C40FD51FEC17FD0761F4808127
:10A1500091810296840F951FE901998388838281FA
:10A1600093819B838A83F0E0E0E012968D919C912D
:10A1700013970097B9F52D913C911197CD01029657
:10A18000820F931F20911508309116082817390760
:10A1900039F6309751F51092180810921708B093BD
:10A1A0001608A0931508BCCFD383C2834081518188
:10A1B000840F951FC817D90761F44E5F5F4F8881E0
:10A1C0009981480F591F518340838A819B819383D2
:10A1D00082832115310509F0B0CFF0931808E09380
:10A1E00017089ECFFD01DC01C0CF13821282D7CFAA
:10A1F0004F925F926F927F928F929F92AF92BF9297
:10A20000CF92DF92EF92FF920F931F93CF93DF9342
:10A210008C01009799F4CB01DF91CF911F910F91A1
:10A22000FF90EF90DF90CF90BF90AF909F908F9076
:10A230007F906F905F904F900C94D34FFC01E60F8E
:10A24000F71F9C0122503109E217F30708F4AEC052
:10A25000D901CD91DC911197C617D70720F1C530F0
:10A26000D10578F0CE0104978617970750F0C61BEA
:10A27000D70B2297C193D1936D937C93CF010E940A
:10A280006F50C801DF91CF911F910F91FF90EF9018
:10A29000DF90CF90BF90AF909F908F907F906F9006
:10A2A0005F904F9008955B01AC1ABD0A4C018C0E73
:10A2B0009D1EA0911708B0911808512C412CF12C2B
:10A2C000E12C109731F580911508909116088815AA
:10A2D000990509F05CC04616570608F058C08091F1
:10A2E000000190910101009741F48DB79EB7409114
:10A2F000040150910501841B950BE817F90708F03C
:10A3000055C0F0931608E0931508F9017183608336
:10A31000B8CF8D919C91119712966C9012971396CD
:10A320007C901397A815B90559F56C0142E0C40E4D
:10A33000D11CCA14DB0420F1AC014A195B09DA0113
:10A340001296159780F06282738251834083D901FF
:10A350006D937C93E114F10471F0D7011396FC9393
:10A36000EE9312978ECF22968C0F9D1FF901918349
:10A370008083F301EFCFF0931808E093170881CFA3
:10A380004816590608F42C017D01D3019ACFCB0160
:10A390000E94D34F7C01009749F0AE01B8010E94A2
:10A3A000FB51C8010E946F5087016BCF10E000E0A5
:10A3B00068CF81E090E0F8940C947055FB01DC01CB
:10A3C00005900D920020E1F70895FC010590002012
:10A3D000E9F7809590958E0F9F1F0895FB01DC0192
:10A3E00004C08D910190801921F441505040C8F76C
:10A3F000881B990B0895FB01DC0102C001900D92AE
:10A4000041505040D8F70895DC0101C06D93415090
:10A410005040E0F70895FC018191861721F08823D0
:10A42000D9F7992708953197CF010895FB01DC01F1
:10A430008D91019080190110D9F3990B0895FB01BA
:10A44000DC0101900D920020E1F70895FB01DC0191
:10A450004150504048F001900D920020C9F701C0D2
:10A460001D9241505040E0F70895FB015191552352
:10A47000A9F0BF01DC014D9145174111E1F759F4F5
:10A48000CD010190002049F04D9140154111C9F3D3
:10A49000FB014111EFCF81E090E001970895453233
:10A4A000510520F4423010F00C945A52FB011082F6
:10A4B000CB010895BB27FB015527AA27880F991FB9
:10A4C000AA1FA41710F0A41B83955051B9F7A05DE3
:10A4D000AA3308F0A95DA193009779F7B111B19360
:10A4E0001192CB010C94BD540F931F93CF93DF9324
:10A4F000CDB7DEB72E970FB6F894DEBF0FBECDBF37
:10A500000D891E8986E08C831A8309838FEF9FE76C
:10A510009E838D83AE01475E5F4F6F89788DCE013C
:10A5200001960E94A4522F813885020F131FF80153
:10A5300010822E960FB6F894DEBF0FBECDBFDF910E
:10A54000CF911F910F9108952F923F924F925F925A
:10A550006F927F928F929F92AF92BF92CF92DF9233
:10A56000EF92FF920F931F93CF93DF93CDB7DEB798
:10A570002B970FB6F894DEBF0FBECDBF7C013B0119
:10A580008A01FC0117821682838181FFDDC1CE0121
:10A5900001965C01F7019381F30193FD859193FF8F
:10A5A00081913F01882309F453C1853239F493FD29
:10A5B000859193FF81913F01853229F4B70190E0A5
:10A5C0000E94CD54E7CF912C212C312CFFE1F315C3
:10A5D00038F08B3211F190F4803209F1833229F195
:10A5E00037FC3CC020ED280F2A3050F536FE20C045
:10A5F0008AE0989E200D1124922E06C08D3291F093
:10A60000803371F7689430F8F30193FD859193FFDF
:10A6100081913F018111DACF21C0689431F86894AB
:10A6200032F8F2CF689433F8EFCF689434F8ECCF77
:10A63000EAE02E9E200D1124222E689435F8E4CFF6
:10A640008E3229F436FC04C1689436F8DDCF8C369E
:10A6500019F4689437F8D8CF8836B1F2982F9F7DD7
:10A6600095549330E0F08336A1F18337C1F18335FF
:10A6700009F063C02801F2E04F0E511CF801C080C0
:10A68000D180692D70E036FC02C06FEF7FEFC6010C
:10A690000E94A7544C01689437F882010AC00C5FED
:10A6A0001F4FFFE3F98388248394912C6501E8947C
:10A6B00037F833FE2DC0522C8114910471F55520CA
:10A6C00009F468CFB70180E290E00E94CD545A941B
:10A6D000F6CFF801808189830E5F1F4FE4CF2801F8
:10A6E000F2E04F0E511CF801C080D180692D70E05E
:10A6F00036FC02C06FEF7FEFC6010E94B2544C01DE
:10A700008201D5CFB70180E290E00E94CD542A9417
:10A710002814190409F0B0F7CECFF60137FC859163
:10A7200037FE81916F01B70190E00E94CD54511026
:10A730005A94F1E08F1A9108BFCF843619F0893608
:10A7400009F077C0F80137FE6BC0608171818281AA
:10A7500093810C5F1F4FF32DFF763F2E97FF09C0AB
:10A7600090958095709561957F4F8F4F9F4F68941E
:10A7700037F82AE030E0A5010E94FD54C82ECA181F
:10A780008C2C432C36FE0CC0E89440F8C91440F4DD
:10A7900034FE05C032FC03C0F32DFE7E4F2E892C03
:10A7A00044FEAAC0FE01EC0DF11D8081803309F04A
:10A7B0009CC0242D297E422E842D8870582E43FC67
:10A7C000AAC040FEA4C09C2C821418F42C0C922C1D
:10A7D000981844FEA6C0B70180E390E00E94CD54D3
:10A7E00042FE09C088E790E041FE02C088E590E0A3
:10A7F000B7010E94CD54C91408F49FC0CA94D12C4B
:10A800009FEFC91AD90ACA0CDB1CF60182916F01AD
:10A81000B70190E00E94CD54AC14BD04B1F74FCF06
:10A8200060817181072E000C880B990B0E5F1F4F02
:10A8300092CFD32CE894D4F82AE030E08537E1F1C8
:10A84000232D297FD22E8F36A9F1F0F4883551F1CE
:10A85000F701868197812B960FB6F894DEBF0FBE65
:10A86000CDBFDF91CF911F910F91FF90EF90DF90BF
:10A87000CF90BF90AF909F908F907F906F905F90A0
:10A880004F903F902F900895803749F0883701F717
:10A89000D4FE02C06894D2F820E130E00DC0689484
:10A8A000D4F8F6CF34FE03C0822F8660D82E20E184
:10A8B00032E002C028E030E0F801D7FE0FC060812E
:10A8C0007181828193810C5F1F4FA5010E94FD540D
:10A8D000C82ECA183D2CE89437F852CF6081718198
:10A8E00090E080E00E5F1F4FF0CF42FC02C08394E7
:10A8F00063CF8394839460CF842D867809F45CCFF2
:10A90000F6CFB70180E290E00E94CD548394821488
:10A91000C0F3512C5ECF522C5818821408F459CF32
:10A92000F8CF842D867809F466CF8BE241FE80E271
:10A9300047FC8DE2B70190E05CCFB70180E390E087
:10A940000E94CD549A9457CF8FEF9FEF84CFFC0194
:10A950000590615070400110D8F7809590958E0F4A
:10A960009F1F0895FC016150704001900110D8F7BD
:10A97000809590958E0F9F1F0895DC01FC01672F35
:10A9800071917723E1F7329704C07C916D937083C6
:10A990006291AE17BF07C8F308950F931F93CF932B
:10A9A000DF93182F092FEB018B8181FD09C01FEF69
:10A9B0000FEF812F902FDF91CF911F910F9108956D
:10A9C00082FF14C02E813F818C819D812817390719
:10A9D0003CF4E881F981CF01019699838883108343
:10A9E0008E819F8101969F838E83E3CFE885F985D1
:10A9F000812F0995892BA1F3DACFFA01AA272830F4
:10AA000051F1203181F1E8946F936E7F6E5F7F4F3B
:10AA10008F4F9F4FAF4FB1E03ED0B4E03CD0670FB7
:10AA2000781F891F9A1FA11D680F791F8A1F911D0A
:10AA3000A11D6A0F711D811D911DA11D20D009F45A
:10AA400068943F912AE0269F11243019305D31939C
:10AA5000DEF6CF010895462F4770405D4193B3E085
:10AA60000FD0C9F7F6CF462F4F70405D4A3318F02C
:10AA7000495D31FD4052419302D0A9F7EACFB4E0DD
:10AA8000A6959795879577956795BA95C9F7009795
:10AA90006105710508959B01AC010A2E0694579536
:10AAA000479537952795BA95C9F7620F731F841F8D
:10AAB000951FA01D0895E199FECF9FBB8EBBE09A24
:10AAC00099278DB30895262FE199FECF9FBB8EBBAA
:10AAD0002DBB0FB6F894E29AE19A0FBE0196089545
:10AAE00018E0CEE1D8E004C0FE010E94B04F2196EC
:0AAAF000CF31D107C9F7F894FFCF6A
:10AAFA00000019088000FFFF01001A01FFFFFFFF95
:10AB0A002A2A2A2A2A2A2A2A2A2A2A2A005B005D8B
:10AB1A00002020286C2D002C20682D002C20642D6C
:10AB2A000029002020202020202020202020202052
:10AB3A002020200025303258002530345800313684
:10AB4A000032340073746172745F6164722D006C38
:10AB5A00656E5F6164722D00656E645F6164722D5B
:10AB6A00002E524B002E524B52002E524B4F002EAB
:10AB7A00425255002E524B4D002E524B50002E522F
:10AB8A004B41002E524B53002E524B49002E42533A
:10AB9A004D002E425353002E45444D002E47414D41
:10ABAA00002E4D4B002E544150002E545A58002E60
:10ABBA0054000A0A00203C3C3C2000203E3E3E0055
:10ABCA002F2E2E002053544F5020504C41590066CE
:10ABDA00696C655F6E616D65202D20002F00496EDE
:10ABEA007365727420534420434152442020004E1E
:10ABFA006F2053442063617264003C3C506C61795D
:10AC0A0065723E3E0000000000361E5C1E4C1E7936
:10AC1A001E3B1F991EA31E00000000BA2C404BA722
:10AC2A00284E0800000000FD332C344B08C6339D23
:10AC3A0033A433B73300000000F53D404B4B084EB8
:10AC4A00087B4F3E373F375E374637523791363E9D
:10AC5A00371A39A1386E37A737E0372538A2384274
:10AC6A003800000000F53D404B4B084E08E63E3EDA
:10AC7A00373F375E374637523791363E371A394CA7
:10AC8A004086444A44E0372538A23842380000005A
:10AC9A00004547404B4B084E0800000000044A405C
:0EACAA004B9849E4496A49844976490D0A00ED
:00000001FF
